:100000000C94EB0BFFFFFFFFFFFFFFFFFFFFFFFF66
:10001000FFFFFFFFFFFFFFFFFFFFFFFFFFFFFFFFF0
:10002000FFFFFFFFFFFFFFFFFFFFFFFFFFFFFFFFE0
:10003000FFFFFFFFFFFFFFFFFFFFFFFFFFFFFFFFD0
:10004000FFFFFFFFFFFFFFFFFFFFFFFFFFFFFFFFC0
:10005000FFFFFFFFFFFFFFFFFFFFFFFFFFFFFFFFB0
:10006000FFFFFFFF0C940208FFFFFFFFFFFFFFFFF2
:100070000C94D207FFFFFFFFFFFFFFFFFFFFFFFF13
:10008000FFFFFFFFFFFFFFFFFFFFFFFFFFFFFFFF80
:10009000FFFFFFFFFFFFFFFFFFFFFFFFFFFFFFFF70
:1000A000FFFFFFFFFFFFFFFFFFFFFFFFFFFFFFFF60
:1000B000FFFFFFFFFFFFFFFFFFFFFFFFFFFFFFFF50
:1000C000FFFFFFFFFFFFFFFFFFFFFFFFFFFFFFFF40
:1000D000FFFFFFFFFFFFFFFFFFFFFFFFFFFFFFFF30
:1000E000FFFFFFFFFFFFFFFF0C946E07FFFFFFFF07
:1000F000FFFFFFFFFFFFFFFFFFFFFFFFFFFFFFFF10
:10010000FFFFFFFFFFFFFFFFFFFFFFFFFFFFFFFFFF
:10011000FFFFFFFFFFFFFFFFFFFFFFFFFFFFFFFFEF
:10012000FFFFFFFFFFFFFFFFFFFFFFFFFFFFFFFFDF
:10013000FFFFFFFF0C946B2FFFFFFFFFFFFFFFFF91
:10014000FFFFFFFFFFFFFFFFFFFFFFFFFFFFFFFFBF
:10015000FFFFFFFFFFFFFFFFFFFFFFFFFFFFFFFFAF
:100160000C94E407FFFFFFFFFFFFFFFF0C94A907BC
:10017000FFFFFFFFFFFFFFFFFFFFFFFFFFFFFFFF8F
:10018000FFFFFFFFFFFFFFFFFFFFFFFFFFFFFFFF7F
:10019000FFFFFFFFFFFFFFFFFFFFFFFFFFFFFFFF6F
:1001A000FFFFFFFFFFFFFFFFFFFFFFFFFFFFFFFF5F
:1001B000FFFFFFFFFFFFFFFFFFFFFFFFFFFFFFFF4F
:1001C000FFFFFFFFFFFFFFFFFFFFFFFFFFFFFFFF3F
:1001D000FFFFFFFFFFFFFFFFFFFFFFFF0C94200863
:1001E000FFFFFFFFFFFFFFFFFFFFFFFFFFFFFFFF1F
:1001F000FFFFFFFFFFFFFFFFFFFFFFFFFFFFFFFF0F
:1002000000080404000C020A060E010905000101A1
:1002100002000103040001010400010108000118AB
:1002200018DC0900025353E9093535EB09000201D6
:10023000010202000201160A210A01000C00040159
:10024000690A7B0A900AA50A030000000200000D5B
:100250004E657420616464726573733A20003031B6
:10026000323334353637383941424344454600004D
:10027000010002000400080010002000400080007F
:10028000000100020004000800100020004000806F
:100290000930810E850E890E8D0E910E950E990EE8
:1002A0009D0EA10E080101BD0E0202C10E0404C57F
:1002B0000E0808C90E1010CD0E2020D10E4040D5DA
:1002C0000E8080D90E001030304F0F3131530F3275
:1002D00032570F33335B0F34345F0F3535630F36CE
:1002E00036670F37376B0F38386F0F3939730F4157
:1002F00041770F42427B0F43437F0F4444830F45B6
:1003000045870F46468B0F000CA0A0DC0F5050E035
:100310000F4B4BE40F3C3CE80F2828EC0F1E1EF05F
:100320000F1414F40F1111F80F0F0FFC0F0C0C0029
:10033000100A0A0410060608100004007910801044
:1003400087108E100500B110B510B910BD10C11086
:10035000020202CC100101D2100006474554564556
:100360005200065B4C494E4B5D00085B4C494E4BBE
:100370004F4B5D00085B4745545645525D0000B148
:10038000D36217A6C4752E9FFD4C3988EA5B5CEDDD
:100390008F3E4BFA982972C3A11065D4B607B809ED
:1003A0006BDAAF1E7CCD962745F4813052E3E455DD
:1003B0003786F3422091CA7B19A8DD6C0EBFC1704D
:1003C00012A3D66705B4EF5E3C8DF8492B9A9D2C9D
:1003D0004EFF8A3B59E8B30260D1A41577C679C8AD
:1003E000AA1B6EDFBD0C57E6843540F1932225949D
:1003F000F6473283E1500BBAD8691CADCF7E338209
:10040000E0512495F7461DACCE7F0ABBD9686FDE5C
:10041000BC0D78C9AB1A41F0922356E785348B3A6C
:1004200058E99C2D4FFEA51476C7B20361D0D7665C
:1004300004B5C07113A2F9482A9BEE5F3D8CF243CC
:100440002190E5543687DC6D0FBECB7A18A9AE1F1C
:100450007DCCB9086ADB803153E2972644F54AFB2C
:1004600099285DEC8E3F64D5B70673C2A01116A71C
:10047000C57401B0D2633889EB5A2F9EFC4D02013E
:1004800001DA140000DE1400020123153015020207
:1004900044156115023039414600020D0D3E3E0003
:1004A000050101F31904040D1A0606241A05053B7B
:1004B0001A0000521A00000000A0504B3C281E14E5
:1004C000110F0C0A06000BFEFEE000030000000006
:1004D00000FD0BFEFEE000030000850100FD0BFEA9
:1004E000FEE000030000650300FD0BFEFEE00003DC
:1004F0000000850300FD0BFEFEE000030000350553
:1005000000FD0BFEFEE000030000150700FD0BFEE2
:10051000FEE000030050121000FD0BFEFEE00003A1
:100520000000151400FD0BFEFEE000030050121841
:1005300000FD0BFEFEE000030000202100FD0BFE8D
:10054000FEE000030000952400FD0BFEFEE000032A
:100550000000502800FD0BFEFEE00003000050509C
:1005600000FD0B00471C4F1C571C5F1C671C6F1CB9
:10057000771C7F1C871C8F1C971C0700B61CBE1C99
:10058000C61CCE1CD61CDE1CE61C0CA0A0C11D5037
:1005900050CD1D4B4BD91D3C3CE51D2828F11D1E9F
:1005A0001EFD1D1414091E1111151E0F0F211E0C06
:1005B0000C2D1E0A0A391E0606451E0001E0EF003A
:1005C000020000E0EF0003000003032525000210F5
:1005D00010202000013039000B0035253C25432533
:1005E0004A25512558255F2566256D2574257B25CF
:1005F000090202B4250808C8250A0AC8250303C849
:10060000250404D4250606E2250707F0250505FE86
:100610002509091F26000902023D260A0A41260370
:10062000034126040445260505492606064D2607EE
:10063000075126080855260909592600044E6F6EF1
:10064000650942616E6420446174610449636F6DA1
:10065000074B656E776F6F640646542D383430064D
:1006600046542D3834370646542D39323009465415
:100670002D313030304D500F46542D323030302037
:1006800040204C61746572054F72696F6E08466C4C
:1006900065782053445207556E6B6E6F776E043148
:1006A00032303004323430300434383030043936AB
:1006B000303005313932303005333834303005359B
:1006C00037363030033030300249461920202020A0
:1006D0002030303030303030303030323030303028
:1006E000303030303B0549463030300E2B30303022
:1006F0003030303130303030303B0C2446412072C5
:1007000065636569766564000C2446432072656301
:1007100065697665640C4E6F2024464520666F75CA
:100720006E640649636F6D3A2003494630024641C4
:1007300003404B56043F42460D03404246043F41AE
:10074000460D0340414602FEFE03E003FD03494619
:100750003B0500000002100500000000000500003D
:10076000000003043F4B560D1045787465726E61AE
:100770006C20706F6C6C696E670000CA9A3B00E178
:10078000F5058096980040420F00A08601001027D2
:100790000000E8030000640000000A000000333C91
:1007A0005645523E20534D2D3820536861636B20CF
:1007B0004D617374657220436F6E74726F6C6C65FB
:1007C00072202876312E3139292034204E6F762040
:1007D00032301076312E313920203034204E6F7671
:1007E00020323000063C534D2D383E0001020203FA
:1007F0000405060706070608BE0AA60E881370172A
:100800003421E02E803EBC4DD8599065409C60EA72
:10081000010008000504040505060607070808008E
:100820000700ED2BF52BFD2B052C0D2C152C1D2C6D
:1008300001010C0003005B2E672E732E10536574AC
:1008400074696E672064656661756C747300044139
:1008500049313B1543757272656E7420636F6E6625
:10086000696775726174696F6E0E526164696F2099
:100870006E756D6265723A200C526164696F207406
:100880007970653A200B4261756420726174653A33
:100890002010526164696F2074696D656F757420F2
:1008A0003D2007456E61626C65640844697361624E
:1008B0006C6564134175746F2062616E64206368B7
:1008C000616E6765203D2011436F6E74726F6C20FE
:1008D0006F6E20555342203D200E49636F6D20619D
:1008E0006464726573733A2009537769746368208E
:1008F000233A0A4D6163726F206D6F64650D446920
:10090000726563742073656C6563740D417578203E
:1009100052532D323332203D20074B656E776F6F77
:100920006405596165737509556E646566696E6520
:10093000641244656661756C7420616E74656E6ED8
:1009400061733A200201723077300C012F31363159
:100950003D3144314B3152315931603167316E3163
:1009600075317C3101010C00030202983304049EAE
:10097000330808C1330001000A0002000001010031
:100980000302022E3404045B3408086934000302B5
:1009900002A6340404B8340808C634000101040077
:1009A0000302020A3504041C3508082A350003082E
:1009B000088935040489350202903500030808D4FB
:1009C000350404D4350202DB35000304045D360827
:1009D000085D360202643600030404B8360808B81D
:1009E000360202BF36000100020003000D3719373E
:1009F0002537030404393708084737020255370002
:100A000001010400030404C9370808D7370202E5CE
:100A1000370003040436380808363802023D38002F
:100A2000030404DB380808EA380202F8380003043B
:100A3000047239080872390202793900030404CCBF
:100A4000390808CC390202D339001A0000E73910FE
:100A500010EA392020EC393030EE392121F03932DA
:100A600032F2393333F4393131F6393434F8393537
:100A700035FA394040FC394141FE396060003A6145
:100A800061023A8080043A8181063A5050083A5116
:100A9000510A3A70700C3A71710E3A9090103A9176
:100AA00091123AA0A0143AA1A1163AB0B0183AB1E6
:100AB000B11A3A00040C0C683A0404703A0808A110
:100AC0003A0202D23A00020404E13A0808E33A008A
:100AD000030404ED3A0808EF3A0202F13A00030475
:100AE00004FD3A0808FF3A0202013B000304043106
:100AF0003B0808333B0202353B00030404473B0834
:100B000008493B02024B3B000304045D3B08085FBD
:100B10003B0202613B00030404733B0808753B027F
:100B200002773B00030404893B08088B3B02028DDB
:100B30003B000304049F3B0808A13B0202A33B00C7
:100B4000030404B53B0808B73B0202B93B000204AA
:100B500004CB3B0202CD3B001A0000653A1010DEC8
:100B60003A2020EA3A3030FA3A21210A3B32321058
:100B70003B3333163B31311C3B3434223B35352873
:100B80003B40402E3B41413E3B6060443B616154F1
:100B90003B50505A3B51516A3B7070703B717180B1
:100BA0003B8080863B8181963B90909C3B9191ACB1
:100BB0003BA0A0B23BA1A1C23BB0B0C83BB1B1D6F3
:100BC0003B000848616D6174696F6E0A507265730D
:100BD00073204155544F043136304D042038304D88
:100BE000042037354D042036304D042034304D0478
:100BF0002033304D042032304D042031374D042055
:100C000031354D042031324D042031304D04202047
:100C1000364D03556E6B0C536861636B204D6173E9
:100C200074657210202020202020202020202020E9
:100C3000202020200D4E6F20726164696F20646156
:100C4000746104204D487A064D6163726F20042060
:100C500020202004416E7420062062757379200BD9
:100C60004E6F20416E74202020202006202020205E
:100C7000202005537745727205204175746F052059
:100C8000204D616E0D436F6E6669677572617469A0
:100C90006F6E0E2045786974207C204D656E7573EB
:100CA000200F41737369676E20416E74656E6E61CB
:100CB000730C53657420416E7420666F72200B4E66
:100CC0006F20416E74656E6E612008416E74656EB2
:100CD0006E6120104E6F2062616E642073656C65DA
:100CE000637465640B536574757020526164696F39
:100CF0000A526164696F20547970650942617564B4
:100D000020526174650C526164696F206E756D626A
:100D1000657207526164696F2023105475726E20EA
:100D200056464F206B6E6F6220746F10746F206791
:100D300065742043492D5620616464720D526164CC
:100D4000696F20506F6C6C696E6707456E61626CED
:100D500065640844697361626C65640D526164691D
:100D60006F2054696D656F75740C43492F5620616F
:100D70006464726573730773657420746F20104127
:100D800075746F2042616E64204368616E67650F01
:100D9000436F6E74726F6C20766961205553420EFA
:100DA000536574204175782052532D3233320F41F0
:100DB00075782052532D3233322054797065074BA9
:100DC000656E776F6F640559616573750F53657450
:100DD0002053776974636820416464720E537769A5
:100DE00074636820416464726573730B4E6F742082
:100DF00070726573656E740E537769746368204111
:100E0000646472203D200B536574204F70204D6F39
:100E100064650E4F7065726174696E67204D6F6412
:100E200065064D6163726F73085374616E6461721D
:100E3000640D436F6E6669672052656C6179730B50
:100E400052656C61797320666F72200C4155544F66
:100E500020746F20657869740652656C617920068C
:100E6000203D204F464606203D20204F4E10526523
:100E70007365742052656C6179204461746111520C
:100E80006573657420416C6C2052656C6179733FA9
:100E90001059455320285072657373204155544FA3
:100EA000290F4E4F20285072657373204155544FBF
:100EB0002910526573746F72652044656661756CA4
:100EC00074730F436C6561722073657474696E6727
:100ED000733F09537769746865733A200F931F93C2
:100EE0004F935F93EF93FF930FB70F93C3D6008198
:100EF0000170013089F4E0913920F0913A200081AD
:100F00000F9300E011E04F915527042B152B009310
:100F10000120109302200AC0E0913920F0913A207C
:100F200000811127009301201093022000910120DD
:100F30001091022000932125109322250E94511424
:100F40000F910FBFFF91EF915F914F911F910F9103
:100F500018950F931F934F935F93EF93FF930FB7E2
:100F60000F93E0913120F091322000810093032013
:100F7000009198280A3039F4009103200093C32887
:100F80000E94661D06C000910320009320250E9448
:100F90008D160F910FBFFF91EF915F914F911F91B0
:100FA0000F9118950F93EF93FF930FB70F93E09165
:100FB0003320F09134200081009304200F910FBF63
:100FC000FF91EF910F9118950F931F934F935F939C
:100FD000EF93FF930FB70F93E0913520F0913620F8
:100FE000008100930520009105200093C3280E94F2
:100FF000661D0F910FBFFF91EF915F914F911F9170
:101000000F9118950F931F934F935F93EF93FF9357
:101010000FB70F93E0913720F091382000810093B3
:101020000620009106200093C3280E94661D0F91A0
:101030000FBFFF91EF915F914F911F910F91189505
:101040000F920F931F932F933F934F935F93EF93C1
:10105000FF930FB70F93E0913B20F0913C2000816C
:1010600000930720009107200093D6260E94AC161B
:101070000F910FBFFF91EF915F914F913F912F9192
:101080001F910F910F9018950091B5200F7040910E
:10109000EB28041709F00895F89400919A28EEE0DF
:1010A000F2E00E94CE28002311F1EDD500810093DB
:1010B000122060D60093E6280091BC204091BD200C
:1010C000042B0093E728EBEBF0E20081073058F0A7
:1010D00051F04091C0200091E728042B4091C1209D
:1010E000042B0093E728D7D500810093E8280091CE
:1010F0009A28E2E1F2E00E94CE280023C1F0CBD58D
:1011000000810093122036D60093E6280091BC207F
:101110004091BD20042B4091C020042B4091C12060
:10112000042B0093E728C0D500810093E8280091A4
:101130009A28E6E1F2E00E94CE28002369F001E05F
:101140000093002004E600932A294091E6280091AC
:10115000E72804270093E728789404E600932A29D7
:1011600000E000932B290895E3E1F1E2FF93EF9370
:10117000009198280E946C2800E50E9427280F9172
:101180001F91E3E1F1E2FF93EF930E940C2800919D
:101190009A280E940A2900E50E9427280F911F9192
:1011A0000091E3280023F1F0E3E1F1E2FF93EF93F4
:1011B0000E940C2801E00E940A2900E50E942728CD
:1011C0000F911F91E3E1F1E2FF93EF930E940C284E
:1011D0000091EA280E940A2900E50E9427280F9121
:1011E0001F9135C0E3E1F1E2FF93EF930E940C28D9
:1011F00000E00E940A2900E50E9427280F911F9114
:101200000091E828003081F4E3E1F1E2FF93EF93ED
:101210000E940C280091E6280E940A2900E50E94FD
:1012200027280F911F9113C0E3E1F1E2FF93EF93A1
:101230000E940C280091E828009312209BD500689A
:101240000E940A2900E50E9427280F911F91009112
:101250009C28002379F0E3E1F1E2FF93EF930E94F1
:101260000C2801E00E940A2900E50E9427280F911E
:101270001F910EC0E3E1F1E2FF93EF930E940C286F
:1012800000E00E940A2900E50E9427280F911F9183
:10129000E3E1F1E2FF93EF930E940C2800919B2879
:1012A0000E940A2900E50E9427280F911F91E3E17F
:1012B000F1E2FF93EF930E940C28009144281091D3
:1012C0004528012F0E940A2900E50E9427280F9136
:1012D0001F91E3E1F1E2FF93EF930E940C2800914C
:1012E00044280E940A2900E50E9427280F911F9197
:1012F000EDE0F1E24091BD224083ECE0F1E24AEF03
:101300004083E0E1F1E243EC408300E00093D62526
:10131000ECE0F1E2A7EDB5E208E510E00E94B627A7
:101320000E942A1B0091ED28002369F001E0009340
:10133000D625ECE0F1E2A7EDB5E208E510E00E9469
:10134000B6270E942A1B04E100932B2908950091DF
:10135000BC20013031F401E000939C2800E00093B0
:10136000E92808950091BC200130F1F40091BD20DE
:10137000EAE1F2E00E94CE280023B1F00091E328D8
:10138000002341F00091BD200093EA2801E0009382
:101390009C2807C00091BD200093E42800E0009342
:1013A0009C2800E00093E92808950091BA200330BA
:1013B00049F40091B82002C067DE04C0EEE1F2E01B
:1013C0000E9499280091BA20013059F40091B82068
:1013D00004C0BDDF06C0C6DF04C0E4E2F2E00E9444
:1013E0009928089500919828023099F00091982842
:1013F0000093C528009146280093C62800914428F0
:10140000109145280093C7281093C8280E94561EA3
:1014100027C000919828EEE2F2E00E94CE280F93B8
:101420000F910023E9F00091972816C000914428FD
:10143000109145280093CB281093CC280E94DC1EE5
:101440000FC000914428109145280093C92810939B
:10145000CA280E942C1F04C0E4E3F2E00E94B628D0
:1014600000919B28EAE3F2E00E94CE280E94BE276A
:1014700019F000E000939B2800919828003041F07B
:1014800000919C28002321F018D400810093E428C7
:101490000091E4280093102062D400930C20009166
:1014A0000C20003019F40FEF00930C200091E3287A
:1014B0000E94BE270F9340E00091EB280E94D327A3
:1014C000402F0F910423002309F499C000919A281A
:1014D0004EC0E3E1F1E2FF93EF93E8E4F2E00E9413
:1014E000182800910C200E94172900E50E94272847
:1014F0000F911F9140C0E3E1F1E2FF93EF9300E011
:1015000040910C200E946528ECE4F2E00E9418282B
:101510000E94F62800E50E9427280F911F912BC0FA
:10152000E3E1F1E2FF93EF93ECE4F2E00E9418288C
:1015300000910C200E940A2900E00E940A2900E57F
:101540000E9427280F911F9116C0E3E1F1E2FF935B
:10155000EF93E8E4F2E00E94182800910C200E942A
:101560000A2900E50E9427280F911F9104C0EEE38D
:10157000F2E00E94B628EDE0F1E240917C23408346
:10158000ECE0F1E20091EB28005E402F4083E0E1C7
:10159000F1E241E1408300E00093D625ECE0F1E286
:1015A000A7EDB5E208E510E00E94B6270E942A1BCD
:1015B00002E00093D625ECE0F1E2A7EDB5E208E504
:1015C00010E00E94B6270E942A1B00E00093D62557
:1015D000ECE0F1E2A7EDB5E208E510E00E94B627E5
:1015E0000E942A1B02E00093D625ECE0F1E2A7ED71
:1015F000B5E208E510E00E94B6270E942A1B009180
:10160000E3280E94BE2709F46FC0E3E1F1E2FF93F3
:10161000EF9300919A280E946C2800E50E942728E9
:101620000F911F91E3E1F1E2FF93EF930E940C28E9
:101630004CD3019110810E940A2900E50E942728BD
:101640000F911F91E3E1F1E2FF93EF930E940C28C9
:101650003CD301911081012F0E940A2900E50E94CC
:1016600027280F911F91EDE0F1E24091BD224083C8
:10167000ECE0F1E241E34083E0E1F1E247E5408361
:1016800000E00093D625ECE0F1E2A7EDB5E208E535
:1016900010E00E94B6270E942A1B02E00093D62584
:1016A000ECE0F1E2A7EDB5E208E510E00E94B62714
:1016B0000E942A1B00E00093D625ECE0F1E2A7EDA2
:1016C000B5E208E510E00E94B6270E942A1B02E05E
:1016D0000093D625ECE0F1E2A7EDB5E208E510E0D5
:1016E0000E94B6270E942A1B009144281091452889
:1016F000012F00930A200091442800930B20EDE075
:10170000F1E24091BD224083ECE0F1E24AEF4083F8
:10171000E0E1F1E243E14083E3E1F1E2FF93EF93A3
:1017200000919A2840919B280E9465280091EA2800
:101730000093102014D30E940A290091EA280093F4
:1017400010200DD30E940A2900E50E9427280F913E
:101750001F91E3E1F1E2FF93EF930E940C280091C7
:101760000A200E940A2900910B200E940A2900E504
:101770000E9427280F911F9100E00093D625ECE0EE
:10178000F1E2A7EDB5E208E510E00E94B6270E945D
:101790002A1B02E00093D625ECE0F1E2A7EDB5E2CA
:1017A00008E510E00E94B6270E942A1B0091ED2850
:1017B000002369F001E00093D625ECE0F1E2A7ED0B
:1017C000B5E208E510E00E94B6270E942A1B05E159
:1017D0000093E9280895EDE3F0E00FEF402F4083F8
:1017E000EEE3F0E00FEF1FE2012F402F408368D7B8
:1017F0000E94832B00E016E0009375201093762062
:1018000000E000937720009378200EE00093792089
:101810002DD500E216E000937520109376200FEF8F
:101820000093772000E10093782000E00093792076
:101830001DD500E416E000937520109376200AE889
:101840000093772008E80093782000E00093792047
:101850000DD500E616E0009375201093762008E879
:10186000009377200093782000E000937920FED445
:1018700000E816E000937520109376200BEB0093A0
:10188000772008EB0093782000E000937920EED4D5
:1018900000EA16E0009375201093762008E3009389
:1018A00077200FEF0093782000EB00937920DED4AF
:1018B00000E010EA2CE830E0E7E6F0E20E94362A89
:1018C000DFD3E0E0F9E041E04083E1E0F9E040E02F
:1018D0004083E2E0F9E040E04083E3E0F9E040E00B
:1018E0004083E4E0F9E040E04083E6E2F9E049E9E2
:1018F0004083E7E2F9E043E04083E6E0F9E042E0DC
:101900004083009133201091342000936B2010937A
:101910006C2000E011EE22273327EDE6F0E20E9472
:10192000362A03E00093712000E0009372200093B8
:10193000732000937420CED3009131201091322077
:1019400000936B2010936C2000E815E222273327C8
:10195000EDE6F0E20E94362A03E00093712000E0F9
:10196000009372200093732002E000937420B2D39E
:10197000009135201091362000936B2010936C203D
:1019800000E815E222273327EDE6F0E20E94362A2E
:1019900003E00093712000E0009372200093732015
:1019A00002E00093742096D30091372010913820E4
:1019B00000936B2010936C2000E815E22227332758
:1019C000EDE6F0E20E94362A03E00093712000E089
:1019D000009372200093732002E0009374207AD366
:1019E00000913B2010913C2000936B2010936C20C1
:1019F00000E815E222273327EDE6F0E20E94362ABE
:101A000003E00093712000E00093722000937320A4
:101A100002E0009374205ED30091392010913A20A7
:101A200000936B2010936C2000E012EC21E030E07A
:101A3000EDE6F0E20E94362A04E00093712000E017
:101A4000009372200093732002E00093742042D32D
:101A5000E0ECFAE041E5408307E00093A200E5E511
:101A6000F0E044E04083E2E5F0E04BE84083E0E56D
:101A7000F0E049E14083E0E0F2E041E04083E1E072
:101A8000F2E044E04083E2E0F2E042E04083E3E061
:101A9000F2E040E04083E4E0F2E040E0408301E136
:101AA00000937C230E94562A0E940A1D0E94192F2F
:101AB000789404E611270093652010936620F7D2EE
:101AC000F89433D4789404E00093812600E20E94D5
:101AD0006C28E2E8F6E200E50E9430280E94DC195A
:101AE00001E00093D3260E94CB1901E000938126E8
:101AF000EEE9F7E0A2E8B6E200E50E94452A0E947E
:101B0000DC190E94152D0E94D8160E94E0160E9432
:101B1000021D00919A28085E0093BD2204E6112759
:101B20000093652010936620C2D201E000938126C5
:101B300000E20E946C28E2E8F6E200E50E9430280C
:101B40000E94DC1904E000938126EEE9F7E0A2E8A8
:101B5000B6E200E50E94452A0E94DC1901E00093EC
:101B60008126EEE9F7E0A2E8B6E200E50E94452A08
:101B70000E94DC1904E000938126EFE4F2E00E9469
:101B800018280091BD220E944D290E94F628E2E803
:101B9000F6E200E50E9430280E94DC1900E0009384
:101BA00046280E94761601E000939C280E94D330BC
:101BB00078940E945F2D0E948E3101E0002309F489
:101BC00058C000919A28085E0093BD220091EB282E
:101BD000005F00937C230091ED28002321F008ECA6
:101BE0000093B52103C000E00093B52100912D2999
:101BF000002339F00E94493A00E000932E29009317
:101C00002D2900919828013029F4E5E2F6E040E121
:101C1000408304C0E6E2F6E040E140830E9464268F
:101C200000919828013059F0E4E2F6E0FF93EF9339
:101C300056D0C895002D402FEF91FF9140830E9410
:101C4000D61A002309F0B1DB00912929003029F4CC
:101C50000E94E43902E3009329290091E928003029
:101C600009F4C0DB00912B29003009F47DDAA89536
:101C7000A4CF08950091392010913A2041E050E01E
:101C8000040F151F34C000919A2811274BEB50E226
:101C9000040F151F2CC000919A280E5F11274BEBE3
:101CA00050E2040F151F23C000919A280C5F1127E2
:101CB0004BEB50E2040F151F1AC000919B2811270F
:101CC0004EEE58E2040F151F12C000919B281127F9
:101CD000000F111F4BEF58E2040F151F08C00091B1
:101CE0009B28112740E052E0040F151F00C0E02F91
:101CF000F12FE093E128F093E228089500910E205F
:101D000024C000E000930D2027C001E000930D20C7
:101D100023C002E000930D201FC004E000930D20BB
:101D20001BC008E000930D2017C000E100930D20B8
:101D300013C000E200930D200FC000E400930D20BB
:101D40000BC000E800930D2007C0E0E9F2E00E941C
:101D5000B62800E000930D2000910D200895009119
:101D60001020006300930E20C9DF00930F20009124
:101D70000F2008950091122020C001E0009311204F
:101D800023C002E0009311201FC003E00093112044
:101D90001BC004E00093112017C005E00093112040
:101DA00013C006E0009311200FC007E0009311203C
:101DB0000BC008E00093112007C0E4EAF2E00E94A3
:101DC000992800E00093112000911120089500E06F
:101DD00000932420009114200170013019F400E8D0
:101DE00000932420009114200270023029F4009105
:101DF0002420005C009324200091142004700430FF
:101E000029F400912420005E0093242000911420E6
:101E10000870083029F400912420005F00932420EA
:101E2000009114200071003129F400912420085FF2
:101E300000932420009114200072003229F40091B4
:101E400024200C5F0093242000911420007400349F
:101E500029F4009124200E5F009324200091142087
:101E60000078003829F4009124200F5F009324208B
:101E700000912420009313200091132008950091D5
:101E800016200F7000931620EBD0C895002D0093FC
:101E900015200091152008950091182040C000E001
:101EA0000093172043C001E0009317203FC002E0D9
:101EB000009317203BC003E00093172037C004E0D5
:101EC0000093172033C005E0009317202FC006E0D1
:101ED000009317202BC007E00093172027C008E0CD
:101EE0000093172023C009E0009317201FC00AE0C9
:101EF000009317201BC00BE00093172017C00CE0C5
:101F00000093172013C00DE0009317200FC00EE0C0
:101F1000009317200BC00FE00093172007C0E6ECDA
:101F2000F2E00E94992800E000931720009117200A
:101F3000089500911A2000931820AEDF44E00E941B
:101F400072280F9300911B2000931820A5DF402FCB
:101F50000F91042B0093192000911920089500E09F
:101F60000093272001E000932620009126200830CE
:101F700009F0A8F400911D200170013029F4E7E276
:101F8000F0E200810395008300911D2006950093E7
:101F90001D20E6E2F0E2008103950083E6CF009188
:101FA000272000931C2000911C20089500E000933E
:101FB0001E2000911F2030C001E000931E2030C081
:101FC00002E000931E202CC003E000931E2028C0D6
:101FD00004E000931E2024C005E000931E2020C0D2
:101FE00006E000931E201CC007E000931E2018C0CE
:101FF00008E000931E2014C009E000931E2010C0CA
:102000000AE000931E200CC00BE000931E2008C0C5
:102010000CE000931E2004C0E8E0F3E00E94992841
:1020200000911E20089500912120002321F001E05D
:102030000093202003C000E0009320200091202086
:10204000089500912320003021F400E00093222025
:1020500003C001E000932220009122200023089574
:102060000091162011274EE552E0040F151F00C005
:10207000E02FF12FE093E128F093E22808950895EE
:10208000E7E6F0E20E94312AEBE2F0E20E94362A13
:10209000089540E050E00091292010912A200E94EC
:1020A000E62721F0E9E2F0E20E9405280895009178
:1020B0006520109166200093292010932A2040E08B
:1020C00050E00091292010912A200E94E62709F073
:1020D000F6CF089503E010E040916B2050916C2002
:1020E000040F151F0093A7201093A82000917420BF
:1020F0001CC000E0E091A720F091A820008319C047
:1021000000E1E091A720F091A820008312C000E236
:10211000E091A720F091A82000830BC000E3E0919C
:10212000A720F091A820008304C0EAE3F3E00E9416
:10213000B62804E010E040916B2050916C20040F11
:10214000151F0093A7201093A8200CE1E091A72071
:10215000F091A820008303E00093A4200091712057
:1021600014C000E00093A42014C001E00093A42058
:1021700010C002E00093A4200CC003E00093A42050
:1021800008C007E00093A42004C0E4E4F3E00E9448
:10219000B628009173200CC00091A4200062009327
:1021A000A4200AC00091A42000630093A42004C0CE
:1021B000E0E5F3E00E94992800917220013029F4B3
:1021C0000091A42008600093A42005E010E0409155
:1021D0006B2050916C20040F151F0093A7201093C3
:1021E000A8200091A420E091A720F091A8200083CE
:1021F00006E010E040916B2050916C20040F151FF9
:102200000093A7201093A82048E050E060E070E021
:10221000EDE6F0E20E94312A0E9424270E94402A23
:10222000EBE2F0E20E94312A0E94682741E050E090
:1022300060E070E00E949E270093A5201093A620E6
:102240000091A520E091A720F091A8200083E7EA63
:10225000F0E20E94FE270091A5201091A620012FF8
:10226000E091A720F091A82000830895E0917520C7
:10227000F0917620409177204083B0D24091782031
:102280004083009179200170013019F4B0D248E107
:102290004083009179200270023019F4B1D248E1F4
:1022A0004083009179200470043019F4B2D248E1DF
:1022B0004083009179200870083019F4B3D248E1C6
:1022C0004083009179200071003119F4B4D248E1C3
:1022D0004083009179200072003219F4B5D248E1B0
:1022E0004083009179200074003419F4B6D248E19B
:1022F0004083009179200078003819F4B7D248E182
:1023000040830895E0E8F0E20E943B2AECE7F0E227
:102310000E94312A0E94682700937A2010937B2024
:1023200000917A2010917B200895EF93FF930F93F3
:102330002F93E0E4F0E008ED23E004BF20832F9129
:102340000F91FF91EF910091CF010078003009F0DB
:10235000FACF0895EF93FF930F932F93EBECF1E0F7
:1023600008ED21E004BF20832F910F91FF91EF91A1
:102370000091CF010078003009F0FACF0895F89469
:102380000091CF010078003009F0FACFEAECF1E0DB
:1023900046E34083DFDFEAECF1E043E34083E2EC35
:1023A000F1E040E04083E1ECF1E0009194201091F5
:1023B0009520012F402F4083E0ECF1E040919420E4
:1023C0004083E4ECF1E0409196204083EAECF1E0B8
:1023D00045E34083BFDF789408950091992000235E
:1023E00069F0009197201091982000939420109309
:1023F00095200BEB00939620C2DF0CC00091972034
:1024000010919820009394201093952000E0009361
:102410009620B5DF0895F8940091CF010078003040
:1024200009F0FACFE0ECF1E0409185204083E1EC47
:10243000F1E00091852010918620012F402F4083EC
:10244000E2ECF1E040E04083EAECF1E046E040837A
:1024500081DF0091C401009384207894009184204E
:102460000895009188201091892000938520109371
:102470008620D1DF0B3B21F401E00093872003C0CD
:1024800000E00093872000918720002308950091A9
:102490008C2010918D200093852010938620BBDF27
:1024A0000093AB2001E010E040918C2050918D20F2
:1024B000040F151F0093852010938620ACDF009336
:1024C000AA2040E051E00091AA2011270E94152780
:1024D000512F402F0091AB201127042B152B009377
:1024E0008A2010938B2000918A2010918B200895D0
:1024F0000CEA10E20093B0201093B12000919220DA
:1025000010919320009385201093862084DFE09122
:10251000B020F091B1200083E0EBF0E20E94FE27B2
:10252000E2E9F0E20E94FE270091922010919320B0
:1025300000938520109386206EDFE091B020F0910B
:10254000B1200083E0EBF0E20E94FE27E2E9F0E236
:102550000E94FE27009192201091932000938520E5
:102560001093862058DFE091B020F091B1200083D5
:10257000E0EBF0E20E94FE27E2E9F0E20E94FE2793
:102580000091922010919320009385201093862033
:1025900042DFE091B020F091B1200083ECEAF0E25C
:1025A0000E94312AEEE8F0E20E94362A00918E2045
:1025B00010918F20209190203091912008950091CA
:1025C0009A2010919B2000939420109395200091C5
:1025D0009C2000939620D3DE01E010E040919A20E9
:1025E00050919B20040F151F009394201093952069
:1025F00000919C2010919D20012F00939620BFDE1A
:10260000089500EA10E20093B2201093B3200091E5
:102610009E2010919F200093942010939520E0918C
:10262000B220F091B320008100939620A8DEE2EB67
:10263000F0E20E94FE27EEE9F0E20E94FE27009100
:102640009E2010919F200093942010939520E0915C
:10265000B220F091B32000810093962090DEE2EB4F
:10266000F0E20E94FE27EEE9F0E20E94FE270091D0
:102670009E2010919F200093942010939520E0912C
:10268000B220F091B32000810093962078DEE2EB37
:10269000F0E20E94FE27EEE9F0E20E94FE270091A0
:1026A0009E2010919F200093942010939520E091FC
:1026B000B220F091B32000810093962060DE08954F
:1026C00000E011270093312010933220112700934E
:1026D0003320109334201127009335201093362097
:1026E00011270093372010933820112700933920A9
:1026F00010933A20112700933B2010933C20112780
:1027000000933D2010933E20112700933F2010930B
:102710004020112700932F20109330201127009381
:10272000412010934220112700934320109344200E
:10273000112700934520109346201127009347202E
:102740001093482011270093492010934A20112705
:1027500000934B2010934C20112700934D20109391
:102760004E20112700934F201093502011270093E3
:10277000512010935220112700935320109354207E
:1027800011270093552010935620112700935720AE
:102790001093582011270093592010935A20112785
:1027A00000935B2010935C20112700935D20109311
:1027B0005E20112700935F20109360201127009363
:1027C00061201093622011270093632010936420EE
:1027D00011270093292010932A2008950091752035
:1027E0001091762044E050E0040F151F48C000917E
:1027F00075201091762040E150E0040F151F3FC076
:10280000009175201091762041E150E0040F151FD2
:1028100036C0009175201091762042E150E0040FFF
:10282000151F2DC0009175201091762043E150E0D6
:10283000040F151F24C0009175201091762044E1EB
:1028400050E0040F151F1BC00091752010917620D9
:1028500045E150E0040F151F12C000917520109142
:10286000762046E150E0040F151F09C00091752045
:102870001091762047E150E0040F151F00C0E02FB3
:10288000F12FE093E128F093E22808950091B6211A
:10289000003030F029F0E6EBF1E200810A95008388
:1028A00008950091BB220F37B0F41BD7409121252A
:1028B0005091222541935083E9EBF2E20081039588
:1028C0000083EBEBF2E20081039500830091B922D3
:1028D0000F770093B9220895F89400E00093B9228D
:1028E0000093BA220093BB227894089500E00093ED
:1028F000D7260093D826EEEBF2E20081043008F4EC
:1029000025C002E00093D926EEEBF2E2408100916F
:10291000D926041709F058F4F6D6C895002D00936F
:10292000D826E9EDF6E2008103950083EDCF009112
:10293000D8264FEF04270093D8260091BF2240915C
:10294000D826041719F401E00093D7260091D72662
:102950000023089500E00093DB2601E01127009397
:10296000DC261093DD26EBEFF2E240815527009143
:10297000DC261091DD260E94F02751F0D8D6C895AC
:10298000002D0093DB26ECEDF6E20E94FE27EBCF54
:102990000091DB264FEF04270093DB260091DB2616
:1029A0000093DA260091DA26089500E00093DE26EF
:1029B00002E008C004E60093B52108C000E00093DF
:1029C000B52104C0EEE7F4E00E9499280091B821F7
:1029D000003010F009F0E1C00091BB22003008F493
:1029E000DCC009F4DAC0F894ADD6019110810093EF
:1029F000DF261093E026EAEBF2E2008103950083E4
:102A0000EBEBF2E200810A9500830091BA220F7786
:102A10000093BA22789440E051E00091DF261091B3
:102A2000E0260E94E62761F001E00093BC22E6EB7D
:102A3000F4E00E941828EEEBF2E20CE30E9430284A
:102A40000091BC221AC040E051E00091DF261091B5
:102A5000E0260E94DE2719F002E00093BC2211C09C
:102A600040E051E00091DF261091E0260E94D62739
:102A700019F003E00093BC2204C0E8E8F4E00E94EF
:102A8000B6280091BC2284C0EEEBF2E2008108324D
:102A9000A0F4EEEBF2E20E940C280FEF10E0409160
:102AA000DF265091E026042315230E940A29EEEB2D
:102AB000F2E20CE30E94302803C000E00093BC2245
:102AC0006BC014DF002309F456C0E5EBF0E200917F
:102AD000C1220083E4EBF0E20091C0220083E8EB26
:102AE000F0E20091C2220083E7EBF0E20091C32202
:102AF0000083EBEBF0E2FF93EF93E6EBF4E00E9450
:102B0000182800E50E9427280F911F9106E00093E6
:102B1000E126EEEBF2E240810091E126041709F094
:102B2000A8F4EBEBF0E2FF93EF930E940C2814D68D
:102B300000810E940A2900E50E9427280F911F9119
:102B4000E1EEF6E2008103950083E3CFE9EBF0E2EA
:102B500040E0408300E00093BC2201E00093DE26C9
:102B6000E6EBF4E00E941828EEEBF2E20CE30E94A0
:102B7000302813C00CC0E6EBF4E00E941828EEEBFE
:102B8000F2E20CE30E94302800E00093BC2204C073
:102B9000EEE8F4E00E94B6281FCF0091DE26002365
:102BA000089540E050E00091392010913A200E94B1
:102BB000D62709F008950091E226002321F0D4D50C
:102BC0004DE1408303C0D0D54CE14083089540E0FF
:102BD00050E000914520109146200E94D62709F030
:102BE00008950091E326002321F0C7D542E04083F9
:102BF00003C0CCD542E040830895E6E2F5E240E030
:102C0000408300912325409124250E94652800914E
:102C100027250E940A29009126250E940A29EAE216
:102C2000F5E20E940C280E94F628EBEFF2E200E8A1
:102C30000E9430288FDE0093E426EBEFF2E20E9440
:102C40000C280091E4260E941729EBEFF2E200E83D
:102C50000E943028789401E00093E326B8DF05E075
:102C6000009330290E94363001E00093E22699DF7C
:102C700000E00093D4260091FD220093D526B0D326
:102C800000E00093D4260091FD220093D526A8D31E
:102C900000E00093E22685DF00E000932F26EBEFB3
:102CA000F2E20E940C28E0E3F6E200E50E94302800
:102CB00057D305E0009330290E94363001E000939D
:102CC000E2266FDF00E00093D4260093D52688D358
:102CD00000E00093E22665DF05E0009330290E94C2
:102CE000363000E00093E32672DF089500E00093A1
:102CF000B9220093BA220093BB220093BC22009316
:102D0000B8210093E32663DF00E00093B521009330
:102D10001E2500931F254CD0089502E300937E23C7
:102D200000937F23009124240F33A0F438D54091E1
:102D300020254083E2E2F4E2008103950083E4E28F
:102D4000F4E2008103950083009122240F73009325
:102D5000222401C02DD0089500911F25002349F0A1
:102D600001E00093D4260091D6260093D52638D3CF
:102D70001EC002E300932724009325240091CC2455
:102D80000F33A0F414D54091D6264083EAECF4E248
:102D9000008103950083ECECF4E20081039500834D
:102DA0000091CA240F730093CA2401C009D008956A
:102DB00000E0009322240093232400932424089508
:102DC00000E00093CA240093CB240093CC24089500
:102DD0000BE544E50E946528009180250E944D295D
:102DE0000E94F628EBEFF2E200E80E943028EBEFB9
:102DF000F2E20E940C2802E50E940A2900917C253B
:102E00000E944D290E94F62800917D250E944D299F
:102E10000E94F628EBEFF2E200E80E943028EBEF88
:102E2000F2E20E940C2808E40E940A2900917F2502
:102E30000E944D290E94F628EBEFF2E200E80E9482
:102E40003028EBEFF2E20E940C280DE40E940A29E0
:102E5000EBEFF2E200E80E943028E3E8F5E20081BF
:102E6000003008F101F101E00093E626E3E8F5E225
:102E700040810091E626041709F0A8F4EBEFF2E296
:102E80000E940C289CD400810E944D290E94F628A3
:102E9000EBEFF2E200E80E943028E6EEF6E2008175
:102EA00003950083E3CFEBEFF2E20E940C280DE5DF
:102EB0000E940A29EBEFF2E200E80E94302800911C
:102EC0007B250130F1F441E002E00E94CA270F9314
:102ED00040E00091B5210E94D327402F0F91042B91
:102EE000002371F000917B2500938126EBEFF2E245
:102EF0000E940C28E2E8F6E200E50E9430285CD24D
:102F00000EC000917B2500938126EBEFF2E20E9438
:102F10000C28E2E8F6E200E50E9430284DD2089540
:102F200000E00093E726EDECF4E20E940C28E2E6D4
:102F3000F3E00E9418280E942E2981F00091E826D3
:102F400000938126EAE6F3E0A2E8B6E200E50E94FB
:102F5000452A32D204E60093B521E9C0EDECF4E253
:102F60000E940C28EAE5F3E00E9418280E942E290E
:102F700061F00091E82600938126EEE9F7E0A2E8EF
:102F8000B6E200E50E94452A17D2EDECF4E200819A
:102F900044E00E94D3270F930091CE244BE50E947A
:102FA000CA27402F0F910423002309F4B7C00091D2
:102FB000CF24023581F5E5EBF0E247E04083E4EB16
:102FC000F0E2FF93EF930091D02400931A20009138
:102FD000D12400931B200E94990F402FEF91FF9165
:102FE0004083E8EBF0E2FF93EF930091D32400934A
:102FF0001A200091D42400931B200E94990F402F87
:10300000EF91FF914083E7EBF0E240E0408309E07D
:103010000093E92643C00091CF240435F1F5E8EB95
:10302000F0E2FF93EF930091D02400931A200091D7
:10303000D12400931B200E94990F402FEF91FF9104
:103040004083E4EBF0E2FF93EF930091D3240093ED
:103050001A200091D42400931B200E94990F402F26
:10306000EF91FF914083E5EBF0E2FF93EF93009146
:10307000D52400931A200091D62400931B200E948F
:10308000990F402FEF91FF914083E7EBF0E240E092
:1030900040830EE00093E92601C049C0EBEBF0E26B
:1030A000FF93EF93E6EBF4E00E94182800E50E94FE
:1030B00027280F911F918BD30081E4E9F4E00E944F
:1030C000CE280F93EDECF4E240810091E9260E94B6
:1030D000D027402F0F9104230023E9F0EBEBF0E21F
:1030E000FF93EF930E940C2872D3008100931A2063
:1030F00076D3008100931B200E94990F0E940A2919
:1031000000E50E9427280F911F910091E9260E5F8C
:103110000093E926D0CF01E00093E726E6EBF4E048
:103120000E941828EDECF4E200E50E94302800919E
:10313000E7260023089500E00093EA260091242466
:10314000003009F473C000912424003008F46EC0EC
:1031500009F46CC0F8944CD300810093EB26E3E2B1
:10316000F4E2008103950083E4E2F4E200810A9531
:103170000083009123240F730093232478940091FB
:10318000B5210030B1F40091B621003010F009F003
:10319000FACF06E00093D4260091EB260093D526C3
:1031A0001FD105E00093D4260091EB260093D5268D
:1031B00017D10091EB260B3549F4E6EBF4E00E94C1
:1031C0001828E0E8F3E200E50E9430280091EB26A1
:1031D0000D30E1F4E0E8F3E20E940C28EDECF4E2BB
:1031E00000E50E94302801E00093E82699DE0023E4
:1031F00019F001E00093EA26E6EBF4E00E941828BB
:10320000E0E8F3E200E50E9430280FC0F894E0E81F
:10321000F3E20E940C280091EB260E940A29E0E8C4
:10322000F3E200E50E94302878948DCF0091EA26E1
:103230000023089500E00093ED260091CC24003097
:1032400009F48AC00091CC24003008F485C009F448
:1032500083C0F894D5D200810093EE26EBECF4E223
:10326000008103950083ECECF4E200810A95008371
:103270000091CB240F730093CB24789400911F25E9
:10328000002379F1E8E2F4E20E940C280091EE2696
:103290000E940A29E8E2F4E200E50E943028009149
:1032A000EE26EAE9F4E00E94CE280F930F91002366
:1032B000B9F001E000938126E8E2F4E20E940C28D4
:1032C000E2E8F6E200E50E94302876D0E6EBF4E092
:1032D0000E941828E8E2F4E200E50E9430283CC091
:1032E0003BC00091EE260B3549F4E6EBF4E00E947A
:1032F0001828E8E2F4E200E50E9430280091EE266A
:103300000D30E1F4E8E2F4E20E940C28EDECF4E286
:1033100000E50E94302802E00093E82601DE002349
:1033200019F001E00093ED26E6EBF4E00E94182886
:10333000E8E2F4E200E50E9430280DC0E8E2F4E2A1
:103340000E940C280091EE260E940A29E8E2F4E28D
:1033500000E50E94302876CF0091ED2600230895E5
:1033600001E00093F026E0E3F6E240810091F026D0
:10337000041709F078F400912F260093D42648D240
:1033800000810093D5262CD0E0EFF6E20081039572
:103390000083E9CF08950091D3260093D4260DE051
:1033A0000093D5261DD00091D3260093D4260AE0A1
:1033B0000093D52615D008950091812600932F26DD
:1033C000E2E8F6E20E940C28E0E3F6E200E50E9463
:1033D0003028C6DF009181260093D326DCDF0895D4
:1033E0000091D42679C040E050E000913120109146
:1033F00032200E94DA2781F00AE000937F2310D266
:1034000000810072003009F4FACFE0913120F09190
:1034100032200091D526008363C040E050E0009147
:103420003320109134200E94DA2769F002D2008103
:103430000072003009F4FACFE0913320F09134208B
:103440000091D52600834CC040E050E00091372029
:10345000109138200E94DA2769F0F4D100810072BF
:10346000003009F4FACFE0913720F0913820009134
:10347000D526008335C040E050E000913520109102
:1034800036200E94DA2769F0E6D100810072003010
:1034900009F4FACFE0913520F09136200091D5263D
:1034A00000831EC040E050E00091392010913A2086
:1034B0000E94DA2781F00AE00093B721D5D100817C
:1034C0000072003009F4FACFE0913920F0913A20EF
:1034D0000091D526008304C0E0EAF4E00E94992818
:1034E000089500E00093F226EAEBF0E240E040832A
:1034F0000091B42040917C23041721F4EAEBF0E220
:1035000043E040830091B4204091BD22041721F490
:10351000EAEBF0E241E040830091B4200A3F21F45D
:10352000EAEBF0E242E040830091BA20003019F06B
:1035300001E00093F2260091F22600230895009105
:10354000B920003091F040E050E000913920109116
:103550003A200E94DA2749F0E4EBF0E2A3E2B5E278
:1035600008E510E00E94B62748DB0091B920013041
:1035700061F001E000937B25E4EBF0E2ACE7B5E21B
:1035800008E510E00E94B62723DC0091B920023044
:1035900061F002E000937B25E4EBF0E2ACE7B5E2FA
:1035A00008E510E00E94B62713DC0895E9EBF0E28D
:1035B00043E6408300E00093D42540E050E00091D2
:1035C000392010913A200E94DA2739F0EED90023F1
:1035D00021F0E9EBF0E240E0408340E050E0009170
:1035E0003120109132200E94DA2759F00091B92041
:1035F000033639F4A0DD002321F0E9EBF0E241E0ED
:1036000040830091B92043E60E94CA270F9340E00F
:1036100050E000913B2010913C200E94DA27402F7F
:103620000F910423002339F005DE002321F0E9EB9C
:10363000F0E242E040830091B920033639F051DFD7
:10364000002319F001E00093D42579DF0091D425FF
:10365000002308950091D625003099F440E050E011
:103660000091392010913A200E94DA2749F0E7EDC5
:10367000F5E2A3E2B5E208E510E00E94B627BDDA64
:103680000DC00091D62500937B25E7EDF5E2ACE770
:10369000B5E208E510E00E94B6279ADB0895ECE059
:1036A000F1E24091B5204083EDE0F1E24091BD228E
:1036B0004083E1E1F1E24091B9204083E0E1F1E2B1
:1036C0004091D5254083009111210093D625ECE04F
:1036D000F1E2A7EDB5E208E510E00E94B627BADFF7
:1036E00008950091B9221127000F111F49EB51E2F3
:1036F000040F151FC2C00091D92611274EEB52E2CC
:10370000040F151FBAC0F7DF40810091D8260427A7
:1037100011274EE753E0040F151FAFC00091DC26C0
:103720001091DD264BEF52E2040F151FA6C0F6DF05
:1037300040810091DB26042711274EE753E0040F58
:10374000151F9BC00091BA221127000F111F49EBD2
:1037500051E2040F151F91C00091E12611274EEB95
:1037600052E2040F151F89C00091392010913A20B0
:1037700044E050E0040F151F80C0009145201091D7
:10378000462045E050E0040F151F77C0009145200A
:103790001091462046E050E0040F151F6EC00091C6
:1037A0002224112741ED53E2040F151F66C000913A
:1037B000CA24112749E754E2040F151F5EC0009187
:1037C000E626112743E855E2040F151F56C0009165
:1037D000E92611274DEC54E2040F151F4EC000914D
:1037E000E9260F5F11274DEC54E2040F151F45C069
:1037F00000912324112741ED53E2040F151F3DC012
:103800000091CB24112749E754E2040F151F35C05E
:103810000091F026112740E356E2040F151F2DC03A
:10382000009131201091322041E050E0040F151F2B
:1038300024C0009133201091342041E050E0040F67
:10384000151F1BC0009137201091382041E050E037
:10385000040F151F12C0009135201091362041E051
:1038600050E0040F151F09C00091392010913A2033
:1038700041E050E0040F151F00C0E02FF12FE0934E
:10388000E128F093E22808950091B02858C0ECE3B5
:10389000F6E0AFE9B8E200E10E94452A5BC0E1E44E
:1038A000F6E0AFE9B8E200E10E94452A53C0EBE43C
:1038B000F6E0AFE9B8E200E10E94452A4BC0E0E53E
:1038C000F6E0AFE9B8E200E10E94452A43C0E8E52E
:1038D000F6E0AFE9B8E200E10E94452A3BC0EFE51F
:1038E000F6E0AFE9B8E200E10E94452A33C0E6E61F
:1038F000F6E0AFE9B8E200E10E94452A2BC0EDE610
:10390000F6E0AFE9B8E200E10E94452A23C0E7E70C
:10391000F6E0AFE9B8E200E10E94452A1BC0E7E803
:10392000F6E0AFE9B8E200E10E94452A13C0EDE8F5
:10393000F6E0AFE9B8E200E10E94452A0BC0E2E6FA
:10394000F5E00E94B628E6E9F6E0AFE9B8E200E16A
:103950000E94452A9F918F91EFE9F8E20E940C287E
:103960008F939F9308950091C22838C0EEE9F6E046
:10397000A1EBB8E200E10E94452A3BC0E3EAF6E091
:10398000A1EBB8E200E10E94452A33C0E8EAF6E084
:10399000A1EBB8E200E10E94452A2BC0EDEAF6E077
:1039A000A1EBB8E200E10E94452A23C0E2EBF6E079
:1039B000A1EBB8E200E10E94452A1BC0E8EBF6E06B
:1039C000A1EBB8E200E10E94452A13C0EEEBF6E05D
:1039D000A1EBB8E200E10E94452A0BC0EAE7F5E05E
:1039E0000E94B628E6E9F6E0A1EBB8E200E10E9409
:1039F000452A9F918F91E1EBF8E20E940C288F936A
:103A00009F93089500E00093F5270093F627009315
:103A1000F727089508E110E0009385201093862091
:103A20000E940B120093982809E110E00093852072
:103A3000109386200E940B12009399280BE110E04E
:103A400000938520109386200E940B1200939A28E1
:103A500000E010E000938520109386200E940B1256
:103A600000933A2801E010E0009388201093892009
:103A70000E943112009347280CE110E0009385204A
:103A8000109386200E940B12009397280DE110E0FE
:103A900000938820109389200E94311200934C28B3
:103AA000B1DF00E00093B6210093432800934B2838
:103AB0000093462800939B280093482800934928A8
:103AC00001E000939C280E94CC2B089509E100930B
:103AD00039280AE00093B6210091F7270F3FA8F498
:103AE0000E94BA264091C3284083E5EFF7E20081A7
:103AF00003950083E7EFF7E20081039500830091CF
:103B0000F5270F7F0093F52701C07CDF0895009112
:103B10003928003030F029F0E9E3F8E200810A9515
:103B200000830091CD28003038F031F0EDECF8E260
:103B300000810A95008321C003E60093CD280091FF
:103B40004A28003030F029F0EAE4F8E200810A95D2
:103B5000008300914B28003030F029F0EBE4F8E2CC
:103B600000810A95008300914328003030F029F04D
:103B7000E3E4F8E200810A95008308950091C428E7
:103B800090C006E000932F26E2EDF4E0A0E3B6E259
:103B900000E50E94452AE4DB88C006E000932F265A
:103BA000EEEDF4E0A0E3B6E200E50E94452AD8DBA2
:103BB0007CC006E000932F26EAEEF4E0A0E3B6E234
:103BC00000E50E94452ACCDB70C006E000932F265A
:103BD000E6EFF4E0A0E3B6E200E50E94452AC0DB90
:103BE00064C006E000932F26E2E0F5E0A0E3B6E231
:103BF00000E50E94452AB4DB58C006E000932F265A
:103C0000EEE0F5E0A0E3B6E200E50E94452AA8DB7D
:103C10004CC006E000932F26EAE1F5E0A0E3B6E20F
:103C200000E50E94452A9CDB40C006E000932F2659
:103C3000E6E2F5E0A0E3B6E200E50E94452A90DB6B
:103C400034C006E000932F26E2E3F5E0A0E3B6E2FD
:103C500000E50E94452A84DB28C006E000932F2659
:103C6000EEE3F5E0A0E3B6E200E50E94452A78DB4A
:103C70001CC006E000932F26EAE4F5E0A0E3B6E2DC
:103C800000E50E94452A6CDB10C006E000932F2659
:103C9000E6E5F5E0A0E3B6E200E50E94452A60DB38
:103CA00004C0EAE8F5E00E94992808950091C5282B
:103CB000013031F40091C6280093C4285FDF7BC037
:103CC000E6ECF4E0A6E5B8E20CE00E94452A00919B
:103CD000C7281091C8280E946629EDE4F8E206E0A2
:103CE0000E943028EDE4F8E20081053068F4EDE44C
:103CF000F8E20E940C2800E30E941729EDE4F8E2A4
:103D000006E00E943028EECF00914E280F700093FD
:103D1000542844E0009154280E94722800935428AB
:103D200000914F280F7000935528EFE5F8E240917D
:103D3000552800915428042B402F4083009150288F
:103D40000F700093542844E0009154280E94722878
:103D500000935428009151280F7000935528EEE5E8
:103D6000F8E24091552800915428042B402F4083BD
:103D7000009152280F700093542844E00091542879
:103D80000E94722800935428009153280F700093CA
:103D90005528EDE5F8E240915428408306E0009371
:103DA0002F26E6E5F8E20E940C28E0E3F6E200E5C3
:103DB0000E943028D5DA08950091CB281091CC28A4
:103DC0000E946629EDE4F8E20FE00E943028EDE45D
:103DD000F8E20E940C28E4ECF6E00E9418280E9409
:103DE000F628EDE4F8E20FE00E943028EDE4F8E276
:103DF00000810B3068F4EDE4F8E20E940C2800E347
:103E00000E941729EDE4F8E20FE00E943028EECF7F
:103E100005E000932F26E8ECF6E0A0E3B6E200E52B
:103E20000E94452A9DDA05E000932F26EDE4F8E292
:103E30000E940C28E0E3F6E200E50E94302890DAC8
:103E400005E000932F26EBECF6E0A0E3B6E200E5F8
:103E50000E94452A85DA08950091C9281091CA2840
:103E60000E946629EDE4F8E20FE00E943028EDE4BC
:103E7000F8E20E940C28E4ECF6E00E9418280E9468
:103E8000F628EDE4F8E20FE00E943028EDE4F8E2D5
:103E90000081083068F4EDE4F8E20E940C2800E3A9
:103EA0000E941729EDE4F8E20FE00E943028EECFDF
:103EB00005E000932F26E5EEF6E0A0E3B6E200E58C
:103EC0000E94452A4DDA05E000932F26EDE4F8E242
:103ED0000E940C28E0E3F6E200E50E94302840DA78
:103EE00005E000932F26EBEEF6E0A0E3B6E200E556
:103EF0000E94452A35DA0895F89444D7008100934A
:103F0000CF28E6EFF7E2008103950083E7EFF7E2C1
:103F100000810A9500837894E8EFF7E2008100348D
:103F200068F4E8EFF7E20E940C280091CF280E9485
:103F30000A29E8EFF7E200E40E9430280091CF2838
:103F40000093CE280091ED280E94BE2741F001E0A9
:103F50000093D4260091CF280093D52641DA009112
:103F6000CE2808950091612800936228009162286C
:103F7000007F44E00E947D280E946029ECE5F8E281
:103F800002E00E943028ECE5F8E20E940C28009143
:103F900062280F700E9460290E94F628ECE5F8E282
:103FA00002E00E943028089500E000934D2800911F
:103FB000F727003008F44CC109F44AC19DDF009393
:103FC0006028009160280A3FB9F404E0009381263C
:103FD000EAEFF6E0A2E8B6E200E50E94452AECD955
:103FE00011DDE7E0F7E00E941828E8EFF7E200E4CF
:103FF0000E9430282DC12BC1009160280D3F09F08F
:1040000026C101E000934E28E8EFF7E240810091DD
:104010004E28041709F0F8F4BDD600810C3FA9F42E
:1040200004E000938126E8E0F7E0A2E8B6E200E5CC
:104030000E94452AC1D9E6DCE7E0F7E0F9D7E8EFCE
:10404000F7E200E40E94302803C1EEE4F8E20081C8
:1040500003950083D9CFE8EFF7E200814AE0A0D7CB
:104060000F93E8EFF7E200814EE09DD7402F0F91CC
:10407000042B002341F0E7E0F7E0DAD7E8EFF7E2BE
:1040800000E4EED7E5C00091F9274EEF86D70F93F5
:104090000091FA274EEF81D7402F0F91042B002378
:1040A000A1F0E7E0F7E0C4D7E8EFF7E200E4D8D703
:1040B000A9DC04E000938126E5E1F7E0A2E8B6E29E
:1040C00000E50E94452A78D9C3C00091FC27ECEB9B
:1040D000F5E00E94CE28002341F0E7E0F7E0A8D702
:1040E000E8EFF7E200E4BCD7B3C00091FB27E0ECB7
:1040F000F5E00E94CE280F930091FD27E6ECF5E055
:104100000E94CE280F934F910F910423002309F4AE
:104110009EC00091FD2745E23DD70F930091FE27F9
:1041200040E03BD7402F0F910423002341F0E7E00C
:10413000F7E07ED7E8EFF7E200E492D789C000917C
:104140003A280F3F91F400E010E000939420109380
:1041500095200091FC27009396200E94BF110091AA
:10416000FC2700933A280E94F935E8EFF7E2008136
:10417000015000935F28E7E0F7E05AD7EFE4F8E258
:104180000CE06ED701E000934E2800914E280430D9
:1041900009F0E0F407D6008100936128E3DEEFE444
:1041A000F8E23AD7ECE5F8E237D70E94F628EFE4D8
:1041B000F8E20CE055D7EFE5F8E200810A950083BC
:1041C000EEE4F8E2008103950083DFCF01E0009385
:1041D0005F2800915F280A3009F030F4EFE5F8E23B
:1041E000008103950083F5CFEFE4F8E20081402FD2
:1041F00001E0EFE4F8E20E94D629E7E0F7E018D703
:10420000E8EFF7E200E42CD7EFE4F8E205D70E94EC
:10421000902926F4002711272227332700933B28D3
:1042200010933C2804E000938126E2E2F7E000D7F7
:1042300000913B2810913C280E946629D7D7E2E8DC
:10424000F6E200E50DD7B8D801E000934D28AFCED7
:1042500000914D280023089500E000934D2800911F
:10426000F727003008F477C009F475C045DE0093E5
:104270005928009159280B3309F06CC003E041E044
:10428000E8EFF7E20E94C229E9E2F7E0D1D6E6D7EB
:1042900041F1E8EFF7E200810C3018F111F1E7E0AD
:1042A000F7E0C6D6EEE4F8E20AE0DAD605E046E04A
:1042B000E8EFF7E20E94C229EEE4F8E20AE0D0D685
:1042C000EEE4F8E2A9D60E94902926F400271127EF
:1042D0002227332700933B2810933C2801E00093CA
:1042E0004D2802E041E0E8EFF7E20E94C229EDE24A
:1042F000F7E09ED6B3D739F1E8EFF7E200810A3054
:1043000010F109F1E7E0F7E093D6EEE4F8E20AE015
:10431000A7D605E046E0E8EFF7E20E94C229EEE406
:10432000F8E20AE09DD6EEE4F8E276D6F9D726F474
:10433000002711272227332700933B2810933C287E
:1043400001E000934D28E7E0F7E072D6E8EFF7E2EE
:1043500000E486D684CF00914D280023089500E024
:104360000093D02800913928003010F009F018C0CF
:104370000091F727003009F413C0E7E0F7E058D6C2
:10438000E8EFF7E200E46CD60091F727003040F048
:1043900039F0B2DD0093D12801E00093D028F4CFAA
:1043A0000091D0280023089500E000934D28D7DF26
:1043B000E5D509F06BC0E8EFF7E20081EEECF5E03F
:1043C000EDD60F930F91002309F460C00091FA27F6
:1043D00040E050E060E071E011272227332734D518
:1043E000EEE4F8E20E94362A0091FB2740E050E01C
:1043F00061E070E011272227332726D5EEE4F8E2AA
:104400000E943B2AA0D5EEE4F8E20E94362A0091F1
:10441000FC2740E051E0112708D522273327EEE49E
:10442000F8E20E943B2A8FD5EEE4F8E20E94362A99
:104430000091FD27112722273327EEE4F8E20E949E
:104440003B2A81D5EEE4F8E20E94362AEEE4F8E257
:104450000E94312A44E05CD6EEE4F8E20E94362A5B
:1044600044E650E060E070E0EEE4F8E2FAD730D5E0
:1044700000933B2810933C28E7E0F7E0D9D5E8EF1C
:10448000F7E200E4EDD501E000934D2800914D28BE
:104490000023089500E000934D2861DF6FD509F0F7
:1044A000AAC0E0E5F8E2FF93EF930091F92744E01A
:1044B00024D61127EF91FF9101931083E2E5F8E2F2
:1044C0000091F9270F70112701931083E4E5F8E2BA
:1044D000FF93EF930091FA2744E00FD61127EF9155
:1044E000FF9101931083E6E5F8E20091FA270F703F
:1044F000112701931083E8E5F8E2FF93EF93009111
:10450000FB2744E0FAD51127EF91FF910193108327
:10451000EAE5F8E20091FB270F7011270193108361
:10452000ECE5F8E2FF93EF930091FC2744E0E5D53A
:104530001127EF91FF9101931083EEE5F8E20091CE
:10454000FC270F70112701931083E2E5F8E2019137
:10455000108140E157E251D400934E2810934F2828
:10456000E4E5F8E20191108148EE53E046D4409131
:104570004E2850914F28040F151F00934E2810937A
:104580004F28E6E5F8E20191108144E650E035D489
:1045900040914E2850914F28040F151F00934E282C
:1045A00010934F28E8E5F8E2019110814AE050E0CD
:1045B00024D440914E2850914F28040F151F00938A
:1045C0004E2810934F28EAE5F8E2019110814091BE
:1045D0004E2850914F28040F151F00933B2810932D
:1045E0003C28E7E0F7E024D5E8EFF7E200E438D52F
:1045F00001E000934D2800914D280023089500E02C
:1046000000934D28ACDEBAD409F047C000E0112772
:1046100022273327EEE4F8E229D70091FB2740E078
:1046200050E061E070E01127222733270DD4EEE43B
:10463000F8E21CD70091FC2740E051E01127F5D3A8
:10464000512F402F66277727EEE4F8E20AD771D47E
:10465000EEE4F8E20BD74091FD2755276627772730
:10466000EEE4F8E2FED665D4EEE4F8E2FFD644E6E6
:1046700050E060E070E0EEE4F8E2F3D629D4009375
:104680003B2810933C28E7E0F7E0D2D4E8EFF7E2CC
:1046900000E4E6D401E000934D2800914D2800236A
:1046A000089500E000934D285ADE68D409F04FC009
:1046B0000091FA2740E050E060E071E011272227E6
:1046C0003327C2D3EEE4F8E2D1D60091FB2740E0D5
:1046D00050E061E070E0112722273327B5D3EEE4E4
:1046E000F8E2C9D630D4EEE4F8E2C0D60091FC2757
:1046F00040E051E0112799D322273327EEE4F8E276
:10470000BAD621D4EEE4F8E2B1D60091FD27112704
:1047100022273327EEE4F8E2AED615D4EEE4F8E231
:10472000A5D648EE53E060E070E0EEE4F8E299D6FA
:10473000CFD300933B2810933C28E7E0F7E078D4F0
:10474000E8EFF7E200E48CD401E000934D280091FB
:104750004D280023089500E000934D280091F7278D
:10476000003008F478C009F476C0C6DB00934F2807
:1047700000914F280B3309F06DC002E041E0E8EFF3
:10478000F7E200D6E8ECF6E053D468D50F93E8EFF3
:10479000F7E2008144E107D4402F0F910423002366
:1047A000F9F0E8EFF7E200810C3121F407E0009323
:1047B0004E2803C006E000934E2805E040914E28A5
:1047C000E8EFF7E2DFD5ACD526F400271127222742
:1047D000332700933B2810933C2801E000934D2899
:1047E00002E041E0E8EFF7E2CDD5EDE2F7E020D4DA
:1047F00035D50F93E8EFF7E200814AE0D4D3402F9C
:104800000F9104230023F9F0E8EFF7E200810C3068
:1048100021F404E000934E2803C003E000934E28E7
:1048200005E040914E28E8EFF7E2ACD579D526F4C3
:10483000002711272227332700933B2810933C2879
:1048400001E000934D28E7E0F7E0F2D3E8EFF7E26C
:1048500000E406D483CF00914D280023089500E0A2
:1048600000934D280091F727003008F498C009F410
:1048700096C042DB00936428009164280D3009F053
:104880008DC0E8EFF7E20081053090F189F103E097
:1048900041E0E8EFF7E276D5E0E3F7E0C9D3DED414
:1048A00039F10091FE27023491F405E000932F26A0
:1048B000E4E3F7E0A0E3B6E200E5E7D50E94B01933
:1048C000E9E3F7E0AEE3B8E204E0DFD511C005E0CC
:1048D00000932F26EDE3F7E0A0E3B6E200E5D5D59F
:1048E0000E94B019E2E4F7E0AEE3B8E204E0CDD50F
:1048F00003E041E0E8EFF7E245D5EEE3F8E28CD3E0
:10490000ADD409F444C0E7E0F7E092D3E3E5F8E280
:1049100000E1A6D304E000934E28E8EFF7E24081DF
:1049200000914E28041709F0B8F444D20081E4ED58
:10493000F5E034D4002351F0E3E5F8E26DD33AD248
:10494000008168D4E3E5F8E200E18AD3EEE4F8E21E
:10495000008103950083E1CFE3E5F8E25DD3E0D485
:1049600026F40027112722273327EFE4F8E27ED52B
:1049700048EE53E060E070E0EFE4F8E272D5A8D2D0
:1049800000933B2810933C2801E000934D28E7E07A
:10499000F7E04ED3E8EFF7E200E462D363CF009193
:1049A0004D280023089500E00093D52840E050E012
:1049B0000091D3281091D428F9D221F000E000937F
:1049C000D52826C001E00093D8280091D8280C30C3
:1049D00009F0F0F4F7D1C895002D3196C895102D47
:1049E000512F402F0091D3281091D428E7D251F0B5
:1049F000F5D1C895002D0093D5280091D8280093B3
:104A00009B2806C0E8EDF8E2008103950083DDCF26
:104A1000409146280091D528041751F000E00093FA
:104A2000E9280091EC28002319F001E000939C286C
:104A30000091D528009346280895D0D70093D9280F
:104A400009E1112700936520109366200E945710FA
:104A5000C5D70093DA284091DA280091D9280417A5
:104A600009F008950091DA284DC006EE14E1009394
:104A70004428109345284FC00AE317E000934428C8
:104A80001093452848C002E41EE000934428109388
:104A9000452841C00EEE1BE10093442810934528A1
:104AA0003AC00DE817E2009344281093452833C01C
:104AB0000FE517E300934428109345282CC006EC1B
:104AC00016E4009344281093452825C009EE12E50A
:104AD00000934428109345281EC00CE611E600936D
:104AE00044281093452817C004E51FE60093442886
:104AF0001093452810C008E114EC0093442810934B
:104B0000452809C0E8EDF5E031D300E01127009316
:104B1000442810934528009144281091452800937B
:104B2000D3281093D4283FDF40E050E00091442880
:104B3000109145284BD219F008EC00934A280895AB
:104B400000E000933D2800914728002309F486C027
:104B500001E0009348280091B621003010F009F0E0
:104B6000FACF0091982877C006E000932F26E6E45C
:104B7000F7E05ED200913A284DD3E9E4F7E058D24D
:104B800035D3E0E3F6E200E56BD20E94B01966C0CF
:104B900005E000932F26EDE4F7E0A0E3B6E200E5A0
:104BA00074D40E94B0195AC00E94021D05E00093FF
:104BB0002F26E1E5F7E0A0E3B6E200E566D40E9427
:104BC000B0194CC00E94021D05E000932F26E1E5BC
:104BD000F7E0A0E3B6E200E558D40E94B0193EC069
:104BE0000E94021D05E000932F26E1E5F7E0A0E317
:104BF000B6E200E54AD40E94B01930C005E0009347
:104C00002F26E7E5F7E0A0E3B6E200E53ED40E94F8
:104C1000B01904E6112700936520109366200E94C6
:104C200057100E94021D05E000932F26EDE5F7E0E6
:104C3000A0E3B6E200E529D40E94B0190FC005E058
:104C400000932F26E3E6F7E0A0E3B6E200E51DD4EB
:104C50000E94B01903C0E0EFF5E06BD20AE00093C8
:104C60004328089500E000939D280091F727003025
:104C700009F426C000919E2820C096D900939D2853
:104C80001FC0EADA00939D281BC0B9DC00939D2861
:104C900017C000DC00939D2813C003DD00939D28FE
:104CA0000FC082DB00939D280BC055DD00939D282B
:104CB00007C0D5DD00939D2803C0E6E1F6E039D2B8
:104CC00000919D280023089500914C28002371F045
:104CD00000914A28003051F400E011270093442845
:104CE000109345280093462800939B28009198280C
:104CF000003009F4089500919828013011F49DDEE8
:104D000038C000914328003009F41ADF0091982838
:104D100000939E28A7DF002361F100913B281091AA
:104D20003C28009344281093452800914428109172
:104D300045280093D3281093D42835DE08EC00933F
:104D40004A28009148281AD189F001E000934928A7
:104D50000EE10093432804E000938126E8E6F7E0A3
:104D6000A2E8B6E200E591D30E94DC1900E00093CE
:104D7000482808950091F527112745EF56E2040FC2
:104D8000151F34C00091F627112745EF56E2040F96
:104D9000151F2CC000914E28112748EF57E2040F31
:104DA000151F24C000915F28112748EF57E2040F18
:104DB000151F1CC000914E28112748EF57E2040F21
:104DC000151F14C00091D828112701501040000F62
:104DD000111F48EF57E0040F151F08C00091D82895
:104DE000112748EB54E0040F151F00C0E02FF12FEE
:104DF000E093E128F093E228089504D00F9215D0B3
:104E00000F9010C0002417FF02C0A4D0039457FFD6
:104E100008C02FEF4227522721E0420F2227521FBE
:104E20000394089500FE089595C00024112480E1A4
:104E30005695479510F4000E111E000F111F8A950C
:104E4000B9F7002D112D089504D00F9219D00F90AD
:104E500014C0002437FF02C083D0039477FF0CC036
:104E60008FEF482758276827782781E0480F882741
:104E7000581F681F781F0394089500FE089570C09E
:104E8000002411242224332480E2769567955795D7
:104E9000479520F4000E111E221E331E000F111F15
:104EA000221F331F8A9589F7002D112D222D332DB6
:104EB000089528E00024001F001C041A08F4040EC2
:104EC00010F4889401C008942A95A9F7001F08954A
:104ED000C0DF0F9202D00F90D0CF042E052A062AF1
:104EE000072A11F180E20024112422243324001F18
:104EF000111F221F331F001C111C221C331C041AFB
:104F0000150A260A370A20F4040E151E261E371E1F
:104F100010F4889401C008948A9549F7001F111F66
:104F2000221F331F402C08950FEF1FEF2FEF3FE795
:104F30000895040F151F261F371F0895041B150B16
:104F4000260B370B0895042B152B262B372B089592
:104F500017FF08952FEF0227122748C037FF089543
:104F60008FEF082718272827382743C0012B09F47B
:104F7000089521912D9301501040F8CF002311F096
:104F80000027089501E0002308950027089501E017
:104F9000002308950417D9F3F8CF0417B1F3F7CF1E
:104FA0000417A8F3F2CF401790F3EFCF04171507BB
:104FB00071F3EBCF0417150741F3E9CF0417150779
:104FC00030F3E3CF4017510710F7DFCF40175107F9
:104FD000F0F2DBCF882717FD839557FD8395089561
:104FE000F9DF80FFEFCF107881F2D1CF0F5F1F4F35
:104FF00008950F5F1F4F2F4F3F4F0895019111915B
:105000000F5F1F4F12930293089501911191015068
:105010001040129302930895EF90FF900191102F8A
:10502000002321F021912F930A95E1F71F934AC0A5
:10503000EF90FF90C8953196002D102F002329F096
:10504000C89531960F920A95D9F71F933BC0ADB71B
:10505000BEB713961D912227A10FB21FED91FC91AF
:10506000EF90FF90ADB7BEB711961D91011710F4E8
:10507000019301C011932227A10FB21F11978A2F0C
:105080009B2F1196112341F0002331F03E91319373
:105090001A9511F00A95D1F710C0EF90FF90ADB7B7
:1050A000BEB711964C915527A40FB51F8A2F9B2F81
:1050B00004C001E0002301C000274FB7F8948DBF62
:1050C0009EBF4FBFFE2DEF2D0994EF90FF900F93E1
:1050D0004F9302E00F93F6CFEF90FF900F9301E014
:1050E0000F93F0CF442309F40895483020F4000FC3
:1050F0004A95E9F7089500270895442309F408958F
:10510000483020F406954A95E9F708950027089558
:10511000442309F40895403238F4369527951795BD
:1051200007954A95D1F7089500271127222733279D
:105130000895C895102D31960020B9F0C895319684
:10514000202DC8953196302D021760F0031709F015
:1051500048F4C8953196202DC895F02DE22F2F9157
:105160002F91099432961A95E8CF0895C895102D7D
:105170003196C895202D3196021B78F0011768F4FE
:105180001127000FE00FF11FC895202D3196C8950B
:10519000E22FF02D2F912F9109940895C895319603
:1051A000102D112381F0C895202D3196C895302DF2
:1051B0003196021730F0031709F018F401E00023CC
:1051C00008951A95EFCF00270895EDB7FEB73396EF
:1051D00020813327E20FF31F3196AE2FBF2F1081AE
:1051E000A10FB31F8A2F9B2F11960895EF90FF9068
:1051F000ECDFAE2FBF2F11961F3F39F0222329F08D
:1052000002910E9313952A95F7CF1E9311978A2F2B
:105210009B2F53CFEF90FF90EDB7FEB731961081E3
:105220001F3F21F02F910F9313951F934BCFEF90BA
:10523000FF90EDB7FEB731961081312F2227E10F95
:10524000F21F319622910083022F3150D8F71F3F71
:1052500019F013951F9336CF108334CFEF90FF9042
:10526000B4DF03D009F425CF27CF8A2F9B2F0197D6
:10527000112371F0222339F01A952A953E9142911B
:105280003417B1F318F08894989408950894089509
:105290002223E1F7189488940895EF90FF9042E05C
:1052A000502F529506D05F93502F03D05F934F93AA
:1052B00009CF5F70505D5A3308F40895595F08951F
:1052C000EF90FF9011272227332705C0EF90FF9022
:1052D0002227332700C0AA27EAE7F7E099E0E894FD
:1052E0008827C895402D3196C895502D3196C89580
:1052F000602D3196C895702D319620DE10F0839583
:10530000FCCF17DE16F0882321F06894805D8F9320
:10531000A3959A9529F7005D0F93A395AF93D2CEED
:10532000EF90FF900027112722273327ADB7BEB794
:105330001196EC91EE2311F19927AE0FB91FE89465
:105340009C919D3219F4EA95689403C09B3211F444
:10535000EA9511979C91905398F09A3088F44AE01E
:105360005527662777278CDD090F9927191F291FD5
:10537000391F1197EA9571F70EF4F2DDE8948FCE9C
:1053800068948DCEEF90FF9022271081442361F026
:10539000002351F0E40FF21F141730F031913F93C6
:1053A000439523950A95C1F72F938CCE8E2F9F2F6F
:1053B0001081F9F00023E9F01417D8F05527E40F15
:1053C000F51F242F200F88F0121778F0AE2FBF2F73
:1053D000A00FB51F212F241B201B101B23953D91CF
:1053E00031932A95E1F7412F4395E82FF92F4A95FC
:1053F00040830895EF90FF908E2F9F2FADB7BEB7DB
:105400001196002369F16C91662351F110815527A3
:10541000E00FF51F2E2E3F2E101720F4712F012FB5
:1054200003950EC0012E001A03947F9111901F92D4
:1054300073957F3F11F00A94C9F7ADB7BEB77F935C
:10544000E22DF32DA70FB51F11960E900192039533
:10545000401710F07A95C9F7E82FF92F0A950083C5
:105460001ECE0191119121913081089501931193E4
:1054700021933083089541915191619170810895F4
:10548000402F512F622F732F0895002371F0C8957C
:10549000202D3196201710F00D9302C02D93022F6E
:1054A000C8950D9231960A95D9F7089501E00093B9
:1054B000982803E00093992801E000939A2800E0DF
:1054C0000093462800939B281127009344281093AB
:1054D00045280093E4280093E5280093E6280093EC
:1054E000E7280093E92801E00093EA280EE110E0A4
:1054F00000938820109389200E9431120093E328A2
:1055000000E210E000938520109386200E940B1289
:105510000093EB280BE310E0009388201093892080
:105520000E9431120093EC280FE110E000938820D4
:10553000109389200E9431120093ED2801E000931E
:105540001729009117290C3009F0A0F519D41F2F45
:105550000E2F00938520109386200E940B1200933B
:10556000182900911829E0E1F8E018DE07DD61F064
:1055700007D41F2F0E2F009394201093952000E046
:10558000009396200E94BF1103D4FF93EF93F8D3AA
:105590001F2F0E2F00938520109386200E940B1240
:1055A000402FEF91FF914083E7E1F9E200810395FD
:1055B0000083C7CFEEEEF8E240E04083089504E0B8
:1055C00000938126ECE3F8E0A2E8B6E200E55DDFB7
:1055D0000E94DC1908E110E00093942010939520BC
:1055E00001E0009396200E94BF1109E110E00093B2
:1055F00094201093952003E0009396200E94BF1101
:105600000AE110E0009394201093952000E00093AD
:1056100096200E94BF110BE110E00093942010939C
:10562000952001E0009396200E94BF1101E010E058
:10563000009397201093982001E0009399200E94F6
:10564000ED1100E210E0009394201093952001E00A
:10565000009396200E94BF110CE110E0009394206B
:105660001093952000E0009396200E94BF110EE158
:1056700010E0009397201093982000E00093992069
:105680000E94ED110BE310E00093972010939820F7
:1056900001E0009399200E94ED110DE110E00093CC
:1056A00097201093982001E0009399200E94ED111B
:1056B0000FE110E0009397201093982000E00093F2
:1056C00099200E94ED1101E00093192900911929F8
:1056D0000C3009F0A0F464D31F2F0E2F00939420F8
:1056E0001093952065D3C895002D009396200E94B5
:1056F000BF11E9E1F9E2008103950083E7CFBCD156
:105700000C940000089500EB19E0009331201093F1
:10571000322000EA18E0009337201093382000EB85
:1057200018E0009333201093342000EA19E000932E
:1057300035201093362000EA1AE0009339201093A8
:105740003A2000EA1BE000933B2010933C2000E845
:1057500016E00093412010934220009345201093BF
:10576000462000E216E000934F2010935020009353
:1057700053201093542000934D2010934E200093FB
:105780004B2010934C200093472010934820009307
:10579000492010934A20089500E000934628009382
:1057A0004328EDE4F8E044DCE8EFF7E200E458DCFD
:1057B0000E94021D00919828E4E1F8E0EFDC0F93CD
:1057C0000F91002321F001E000931A2903C000E0AB
:1057D00000931A290091992838C000EB14E0222781
:1057E0003327EBE1F9E242DE3AC000E619E0222776
:1057F0003327EBE1F9E23ADE32C000EC12E1222776
:105800003327EBE1F9E232DE2AC000E815E2222775
:105810003327EBE1F9E22ADE22C000E01BE4222775
:105820003327EBE1F9E222DE1AC000E016E9222775
:105830003327EBE1F9E21ADE12C000E011EE222775
:105840003327EBE1F9E212DE0AC0E0E2F8E08EDC99
:1058500000E815E222273327EBE1F9E207DE0091A9
:1058600098280230C1F50091352010913620009320
:105870006B2010936C20EBE1F9E2F3DDEDE6F0E252
:10588000F5DD03E00093712000911A290093722046
:1058900000E000937320009374200E946A1000912E
:1058A00037201091382000936B2010936C20EBE18F
:1058B000F9E2D7DDEDE6F0E2D9DD03E000937120F7
:1058C00000E0009372200093732001E000937420A5
:1058D0000E946A1037C00091352010913620009345
:1058E0006B2010936C20EBE1F9E2BBDDEDE6F0E21A
:1058F000BDDD03E00093712000911A29009372200E
:1059000000E00093732001E0009374200E946A106D
:10591000009137201091382000936B2010936C2059
:10592000EBE1F9E29EDDEDE6F0E2A0DD03E00093BD
:10593000712000E000937220009373200093742084
:105940000E946A100091ED280023E9F000913120B7
:105950001091322000936B2010936C2000E011EE28
:1059600022273327EDE6F0E281DD03E0009371208A
:1059700000E0009372200093732002E000937420F3
:105980000E946A101BC000913120109132200093B8
:105990006B2010936C20EBE1F9E263DDEDE6F0E2C1
:1059A00065DD03E00093712000E000937220009316
:1059B000732001E0009374200E946A1000919828DF
:1059C000033059F405E000932F26EEE4F8E0A0E35D
:1059D000B6E200E55ADD0E94B0190895009108066C
:1059E00000931F2944E000911F2987DB00931F29A2
:1059F00000911F290F7000931F2900911F29009308
:105A0000152900911529089500E0009316290091A9
:105A10009B28E0E3F8E0C2DB002319F001E00093EB
:105A20001629009116290023089501E000932029EA
:105A3000009120290C3009F0C0F4C4D1FF93EF93FA
:105A4000CBD11F2F0E2F00938C2010938D200E94FE
:105A50004712512F402FEF91FF9141935083E0E285
:105A6000F9E2008103950083E3CFEBEFF8E200E079
:105A700010E001931083089500E000932129009124
:105A800021290C3009F0D0F4B1D11F2F0E2F009333
:105A90009A2010939B2000E0112700939C201093E4
:105AA0009D200E94DF12ACD100E010E00193108332
:105AB000E1E2F9E2008103950083E1CF089504E07B
:105AC00000938126E3E5F8E0A2E8B6E200E5DDDC3C
:105AD0000E94DC1904E000938126E9E6F8E0A8DAE8
:105AE00000919A28EDDB82DBE2E8F6E200E5B8DA25
:105AF0000E94DC1904E000938126E8E7F8E098DAD8
:105B0000009198280093B0280E94441C6FDBE2E8C3
:105B1000F6E200E5A5DA0E94DC1904E00093812694
:105B2000E5E8F8E085DA009199280093C2280E9400
:105B3000B31C5CDBE2E8F6E200E592DA0E94DC19D5
:105B400004E000932F26E1E9F8E0A0E3B6E200E5E7
:105B50009CDC0E94B01900914C28002361F004E005
:105B600000938126E2EAF8E0A2E8B6E200E58DDCE7
:105B70000E94DC190BC004E000938126EAEAF8E0F9
:105B8000A2E8B6E200E581DC0E94DC1904E00093A3
:105B90002F26E3EBF8E0A0E3B6E200E576DC0E9416
:105BA000B0190091EC28002361F004E000938126F5
:105BB000E2EAF8E0A2E8B6E200E567DC0E94DC1960
:105BC0000BC004E000938126EAEAF8E0A2E8B6E21E
:105BD00000E55BDC0E94DC1904E000932F26E7EC73
:105BE000F8E0A0E3B6E200E550DC0E94B0190091B5
:105BF000ED28002361F004E000938126E2EAF8E05A
:105C0000A2E8B6E200E541DC0E94DC190BC004E02A
:105C100000938126EAEAF8E0A2E8B6E200E535DC86
:105C20000E94DC1904E000938126E9EDF8E000DA37
:105C300000913A2832DBDADAE2E8F6E200E510DA3F
:105C40000E94DC1904E000938126E8EEF8E0F0D928
:105C50000091EB2835DBCADAE2E8F6E200E500DA8B
:105C60000E94DC190091E328002361F004E0009316
:105C70008126E2EFF8E0A2E8B6E200E506DC0E9449
:105C8000DC190BC004E000938126EDEFF8E0A2E8F8
:105C9000B6E200E5FADB0E94DC1904E000932F264F
:105CA000EBE0F9E0A0E3B6E200E5EFDB0E94B0191B
:105CB0000091972824C004E000938126EAEAF8E0E6
:105CC000A2E8B6E200E5E1DB0E94DC1926C004E0B0
:105CD00000938126E9E1F9E0A2E8B6E200E5D5DB30
:105CE0000E94DC191AC004E000938126E1E2F9E089
:105CF000A2E8B6E200E5C9DB0E94DC190EC0E4E3CD
:105D0000F8E034DA04E000938126E7E2F9E0A2E863
:105D1000B6E200E5BADB0E94DC1904E000932F260E
:105D2000E1E3F9E0A0E3B6E200E5AFDB0E94B019E1
:105D300001E000932229009122290C3009F0A0F4FF
:105D400004E000932F2666D00081A7DA00E262DA31
:105D5000E0E3F6E200E584D90E94B019E2E2F9E25C
:105D6000008103950083E7CF04E00093812600E2E1
:105D7000B3D9E2E8F6E200E573D90E94DC19089590
:105D80000091172911274CE350E0040F151F4AC05A
:105D90000091172911274EEE58E2040F151F42C03B
:105DA0000091192911274CE350E0040F151F3AC048
:105DB000009119291127015010404CEE57E0040FB3
:105DC000151F30C0009120291127000F111F4BEF24
:105DD00058E2040F151F26C0009120291127000F3B
:105DE000111F41E250E0040F151F1CC00091212932
:105DF0001127000F111F41E250E0040F151F12C0C0
:105E0000009121291127000F111F4BEF58E2040FB9
:105E1000151F08C00091222911274EEE58E2040FE9
:105E2000151F00C0E02FF12FE093E128F093E22846
:105E3000089500E00093B8210093242900932329BA
:105E4000009327290093B72100934A280093E9285B
:105E50000093B52100932D2900932E2900932F291B
:105E60000895009108064FEF04270E700093312922
:105E700000912D2983D871F1009131290030A9F4C6
:105E800000912E29003081F000912F29083C30F03C
:105E900029F000912E29006800932E2901E000933B
:105EA0002D2900E000932F2915C000912F290A3FCA
:105EB00028F4EFE2F9E200810395008300912F2995
:105EC000053040F039F04091312900912E29042B02
:105ED00000932E2908950F931F934F935F93EF9391
:105EE000FF930FB70F9300912329003030F029F072
:105EF000E3E2F9E200810A9500830091B8210030C5
:105F000030F029F0E8EBF1E200810A95008300917E
:105F10002429003038F031F0E4E2F9E200810A95FA
:105F200000839BC009E0009324290E9449100E942D
:105F3000871D0E9446140091B721003030F029F0EF
:105F4000E7EBF1E200810A95008300917E230030A7
:105F500030F029F0EEE7F3E200810A95008300912A
:105F60007F23003030F029F0EFE7F3E200810A955B
:105F7000008300912C29003030F029F0ECE2F9E2A6
:105F800000810A95008300912929003030F029F022
:105F9000E9E2F9E200810A950083E7E2F9E2008193
:105FA0000A95008300912729003051F40091282997
:105FB0000E94BE2700932829E7E8F6E041E04083ED
:105FC00000912529003038F031F0E5E2F9E2008156
:105FD0000A95008342C009E00093252942DF009121
:105FE0002629003038F031F0E6E2F9E200810A9526
:105FF000008333C009E0009326290091E92800308E
:1060000030F029F0E9EEF8E200810A950083009172
:106010002B29003030F029F0EBE2F9E200810A95FB
:1060200000830091B521003030F029F0E5EBF1E27A
:1060300000810A95008300912A29003038F031F060
:10604000EAE2F9E200810A95008307C000E00093CC
:10605000E6280093E7280093E8280F910FBFFF91EF
:10606000EF915F914F911F910F91189500913029F9
:106070000093232900912329003010F009F0FACF72
:106080000895E6EAF6E040E1408340E24083E3EC35
:10609000FAE040914D2940830091C20A0078003017
:1060A00009F4FACFE5EAF6E040E240830895E5EA34
:1060B000F6E040E14083E6EAF6E040E24083E3ECCC
:1060C000FAE04091502940830091C20A00780030E4
:1060D00009F4FACFE5EAF6E040E240830895009142
:1060E00053290AC000E800934D29CBDF09C000EC1A
:1060F00000934D29C6DF04C0E4E4F9E037D80895E1
:10610000E4E5F9E2408100E1041B00936629009177
:106110006629013000F1F9F042E0009166290E9401
:10612000592700936729009167290030A0F099F062
:10613000E4E5F9E20E940C2800E279D800E26AD88E
:10614000E4E5F9E200E10E943028E7E6F9E20081A7
:106150000A950083E8CF009166290170013059F457
:10616000E4E5F9E20E940C2800E254D8E4E5F9E203
:1061700000E10E94302801E000936529E4E5F9E29E
:10618000408100916529041709F060F40E94E23B08
:106190000081009350298BDFE5E6F9E20081039549
:1061A0000083ECCF089500E300934D296ADF0AE0F5
:1061B000112700936520109366200E94571000E37A
:1061C00000934D295EDF0AE01127009365201093AC
:1061D00066200E94571000E300934D2952DF09E327
:1061E00000934D294EDF04E100934D294ADF06E577
:1061F00000934D2946DF0DE600934D2942DF00E76D
:1062000000934D293EDF0CE000934D293ADF06E074
:1062100000934D2936DF01E000934D2932DF00E87D
:1062200000934D292EDF01E000935329E2ECFBE0BF
:10623000A4E5B9E200E129D952DF00E00093322958
:10624000089502E000935329EBECFBE0A4E5B9E2EA
:1062500000E11BD944DF08950091682954C0E6EDA0
:10626000FBE0A3E3B9E205E010D957C0EBEDFBE09A
:10627000A3E3B9E205E009D950C0E0EEFBE0A3E3F7
:10628000B9E205E002D949C0E5EEFBE0A3E3B9E2DB
:1062900005E0FBD842C0EAEEFBE0A3E3B9E205E08B
:1062A000F4D83BC0EFEEFBE0A3E3B9E205E0EDD8A4
:1062B00034C0E4EFFBE0A3E3B9E205E0E6D82DC08B
:1062C000E9EFFBE0A3E3B9E205E0DFD826C0EEEF9B
:1062D000FBE0A3E3B9E205E0D8D81FC0E3E0FCE0AF
:1062E000A3E3B9E205E0D1D818C0E8E0FCE0A3E3FD
:1062F000B9E205E0CAD811C0EDE0FCE0A3E3B9E2E1
:1063000005E0C3D80AC0EAE4F9E00E94B628E2E159
:10631000FCE0A3E3B9E205E0B8D8089501E00093FA
:106320005329E6E1FCE0A4E5B9E200E1AED8D7DE0E
:1063300002E000935329E2EDF7E0A4E5B9E200E1C1
:10634000A4D8CDDE00ED17E0009365201093662001
:106350000E945710089500E0009332290091982878
:106360000030A1F4E3E2FCE0A9E3B9E200E18DD85A
:1063700001E000935329E9E3F9E20E940C28E4E5E7
:10638000F9E200E10E943028AADE8FC040E050E030
:1063900000914428109145280E94D62759F001E029
:1063A00000935329E4E3FCE0A4E5B9E200E16DD8F1
:1063B00096DE7BC000919B28009368294DDF0091F9
:1063C0009828013071F401E000935329E3E3F9E2E6
:1063D0000E940C28E4E5F9E200E10E9430287FDE0B
:1063E00064C000914428109145280E946629E9E67E
:1063F000F9E200E10E943028E9E6F9E20081009329
:106400007A290EE20E946C2800917A290250E9E66E
:10641000F9E240E10E94FA29E9E6F9E20E940C283B
:10642000E2E4FCE00E9418280E94F628E9E6F9E27E
:1064300000E10E943028E9E6F9E240810CE0041B0B
:1064400000937A2900917A29003098F091F0E9E6DA
:10645000F9E20E940C2800E20E940A29E9E6F9E22A
:1064600000E10E943028EAE7F9E200810A95008302
:10647000E9CFE9E6F9E20E940C28E3E3F9E20E94A1
:106480000C280E94F628E9E6F9E200E10E94302893
:1064900001E000935329E9E6F9E20E940C28E4E5C3
:1064A000F9E200E10E9430281ADE0091E32800237F
:1064B000B1F0E7E4FCE00E9418280091EA280E946D
:1064C00060290E94F628EEE4FCE00E9418280E9451
:1064D000F628E9E3F9E200E10E94302842C0009189
:1064E000E628003049F50091E428009310200E942E
:1064F000AF0E4091E72804230030B1F0E3E5FCE063
:106500000E9418280091E4280E9460290E94F62821
:10651000E8E5FCE00E9418280E94F628E9E3F9E289
:1065200000E10E94302807C0EFE5FCE0A9E3B9E2F2
:1065300000E10E94452A15C0E3E5FCE00E9418280E
:106540000091E6280E9460290E94F628EBE6FCE014
:106550000E9418280E94F628E9E3F9E200E10E946F
:10656000302840E00091EB280E94D3270F9340E0B1
:1065700000912A290E94CA27402F0F91042300234B
:1065800081F0E9E3F9E20E940C28E2E7FCE00E94D6
:1065900018280E94F628E9E3F9E200E10E94302879
:1065A00023C000919C28002381F0E9E3F9E20E94D6
:1065B0000C28E8E7FCE00E9418280E94F628E9E38E
:1065C000F9E200E10E9430280FC0E9E3F9E20E94FD
:1065D0000C28EEE7FCE00E9418280E94F628E9E368
:1065E000F9E200E10E94302802E000935329E9E338
:1065F000F9E20E940C28E4E5F9E200E10E9430286B
:106600006EDD089500E10093322901E000935329E3
:10661000E4E8FCE0A4E5B9E200E10E94452A5FDD80
:1066200002E000935329E2E9FCE00E9418280FE7FA
:106630000E9417290EE70E940A29E4E5F9E200E129
:106640000E9430284CDD089500E20093322901E0D9
:1066500000935329E1EAFCE0A4E5B9E200E10E94DD
:10666000452A3DDDEEDD089501E2009332290091D7
:106670009B28E4E6F9E00E94CE280023F1F1009186
:106680009B2800936829E8DD01E000935329E1EBA2
:10669000FCE00E941828E3E3F9E20E940C280E9423
:1066A000F628E4E5F9E200E10E94302818DD0E94B6
:1066B000EA3B0081003061F402E000935329EEEBE5
:1066C000FCE0A4E5B9E200E10E94452A08DD14C01F
:1066D00002E000935329EAECFCE00E9418280E9493
:1066E000EA3B00810E9460290E94F628E4E5F9E275
:1066F00000E10E943028F3DC17C001E00093532929
:10670000E3EDFCE0A4E5B9E200E10E94452AE7DC04
:1067100002E00093532900E20E946C28E4E5F9E2CC
:1067200000E10E943028DBDC089500917B294BC0FA
:1067300000913229007F0093322949C065D9002396
:10674000F9F00E94EA3B0081003038F031F00E94FD
:10675000EA3B00810A95008304C00E94EA3B48E0BE
:1067600040830E94F23B1F2F0E2F00939420109322
:1067700095200E94EA3B0081009396200E94BF1161
:1067800026C042D90023F1F00E94EA3B0081039524
:1067900000830E94EA3B0081083028F021F00E942B
:1067A000EA3B40E040830E94F23B1F2F0E2F0093F4
:1067B0009420109395200E94EA3B0081009396203C
:1067C0000E94BF1104C0E8E6F9E00E9499280895EC
:1067D00000E30093322901E000935329E4EEFCE04A
:1067E000A4E5B9E200E10E94452A79DC2ADD08959A
:1067F00002E30093322900919828E6E7F9E00E942D
:10680000CE280E94BE2719F000E00093982801E0EE
:1068100000935329E0EFFCE0A4E5B9E200E10E9417
:10682000452A5DDC009198280093B0280E94441C02
:10683000E9E3F9E200E10E94302802E000935329E5
:10684000E9E3F9E20E940C28E4E5F9E200E10E94A4
:10685000302845DC089500917C2949C008E110E00A
:1068600000939420109395200091982800939620EF
:106870000E94BF1100E010E0009394201093952037
:106880000FEF009396200E94BF110E940A1D0091F5
:106890009828EAE7F9E00E94CE280F930F91002391
:1068A00031F000913229007F0093322903C003E3C5
:1068B0000093322920C000919828003021F40AE08A
:1068C0000093982805C0E8E9F8E200810A95008362
:1068D00012C0E8E9F8E2008103950083009198284E
:1068E0000A3020F019F000E00093982804C0E0E896
:1068F000F9E00E949928089503E30093322901E00A
:1069000000935329EBEFFCE0A4E5B9E200E10E941B
:10691000452AE5DB009199280093C2280E94B31C08
:10692000E9E3F9E200E10E94302802E000935329F4
:10693000E9E3F9E20E940C28E4E5F9E200E10E94B3
:106940003028CDDB089500917D292EC009E110E0AB
:1069500000939420109395200091992800939620FD
:106960000E94BF110E940A1D04E30093322920C037
:1069700000919928003021F406E00093992805C081
:10698000E9E9F8E200810A95008312C0E9E9F8E23A
:1069900000810395008300919928063020F019F0BA
:1069A00000E00093992804C0EEE8F9E00E949928DD
:1069B000089501E30093322900919A28ECE9F9E067
:1069C0000E94CE280E94BE2719F001E000939A2869
:1069D00001E000935329E5E0FDE0A4E5B9E200E120
:1069E0000E94452A7CDB02E000935329E2E1FDE0AE
:1069F0000E94182800919A280E9460290E94F62877
:106A0000E4E5F9E200E10E94302869DB0895009195
:106A10007E292EC00BE110E0009394201093952066
:106A200000919A28009396200E94BF110E940A1D8F
:106A300002E30093322920C000919A28013021F40A
:106A400004E000939A2805C0EAE9F8E200810A957B
:106A5000008312C0EAE9F8E2008103950083009107
:106A60009A28043020F019F001E000939A2804C01D
:106A7000E0EAF9E00E949928089501E00093532983
:106A8000EAE1FDE0A4E5B9E200E10E94452A27DB46
:106A900002E000935329EBE2FDE0A4E5B9E200E156
:106AA0000E94452A1CDB0CED15E000936520109335
:106AB00066200E945710089504E30093322901E0F4
:106AC00000935329ECE3FDE0A4E5B9E200E10E9464
:106AD000452A05DB00914728002361F002E000937E
:106AE0005329EAE4FDE0A4E5B9E200E10E94452A69
:106AF000F6DA0BC002E000935329E2E5FDE0A4E5DD
:106B0000B9E200E10E94452AEADA089500917F295E
:106B100019C0009147280E94BE270093472816C03D
:106B200001E010E0009397201093982000914728EF
:106B3000009399200E94ED110E940A1D05E3009325
:106B4000322904C0EEEAF9E00E949928089505E38D
:106B50000093322901E000935329EBE5FDE0A4E521
:106B6000B9E200E10E94452ABADA00914C280023DC
:106B700061F002E000935329EAE4FDE0A4E5B9E204
:106B800000E10E94452AABDA0BC002E000935329D2
:106B9000E2E5FDE0A4E5B9E200E10E94452A9FDAC2
:106BA00008950091802920C000914C280E94BE27A2
:106BB00000934C281DC00DE110E000939720109326
:106BC000982000914C28009399200E94ED110E947A
:106BD0000A1D00919828023009F44FDF00913229F4
:106BE000007F0093322904C0ECEBF9E00E94992861
:106BF000089501E000935329E9E6FDE0A4E5B9E238
:106C000000E10E94452A6BDA02E000935329E6E78F
:106C1000FDE00E94182800913A280E944D290E9408
:106C2000F628E4E5F9E200E10E94302858DA00EDA8
:106C300017E000936520109366200E945710089576
:106C400000E40093322901E000935329EEE7FDE0D0
:106C5000A4E5B9E200E10E94452A41DAF2DA08959A
:106C600001E40093322901E000935329EEE7FDE0AF
:106C7000A4E5B9E200E10E94452A31DA0091EC284E
:106C8000002361F002E000935329EAE4FDE0A4E56B
:106C9000B9E200E10E94452A22DA0BC002E000932B
:106CA0005329E2E5FDE0A4E5B9E200E10E94452AAE
:106CB00016DA08950091812919C00091EC280E94EC
:106CC000BE270093EC2816C00BE310E0009397203A
:106CD000109398200091EC28009399200E94ED11C8
:106CE00000913229007F0093322904C0EAECF9E0D8
:106CF0000E949928089500E80093322901E000934A
:106D00005329EFE8FDE0A4E5B9E200E10E94452A3D
:106D1000E6D997DA089501E80093322901E000935B
:106D20005329EFE8FDE0A4E5B9E200E10E94452A1D
:106D3000D6D90091ED28002361F002E00093532999
:106D4000EAE4FDE0A4E5B9E200E10E94452AC7D9E2
:106D50000BC002E000935329E2E5FDE0A4E5B9E2AF
:106D600000E10E94452ABBD90895009182291BC0E9
:106D70000091ED280E94BE270093ED2818C00FE176
:106D800010E000939720109398200091ED28009335
:106D900099200E94ED110E94CC2B00913229007F96
:106DA0000093322904C0E8EDF9E00E949928089583
:106DB00001E000935329EFE9FDE0A4E5B9E200E129
:106DC0000E94452A8CD93DDA089501E600933229C4
:106DD00001E000935329EEEAFDE0A4E5B9E200E109
:106DE0000E94452A7CD900919728E6EEF9E00E949E
:106DF000CE280E94BE2771F000E0009397280CE196
:106E000010E0009394201093952000E000939620CA
:106E10000E94BF110091972824C002E000935329DB
:106E2000E2E5FDE0A4E5B9E200E10E94452A57D978
:106E30001CC002E000935329EEEBFDE0A4E5B9E2AB
:106E400000E10E94452A4BD910C002E0009353296B
:106E5000E6ECFDE0A4E5B9E200E10E94452A3FD955
:106E600004C0EAEEF9E00E94B62808950091832953
:106E70002EC000919728003021F402E0009397285B
:106E800005C0E7E9F8E200810A95008324C0E7E93C
:106E9000F8E200810395008300919728023020F0EA
:106EA00019F000E00093972816C00CE110E0009361
:106EB00094201093952000919728009396200E948B
:106EC000BF1100913229007F0093322904C0E2EF04
:106ED000F9E00E949928089500E50093322901E025
:106EE00000935329ECECFDE0A4E5B9E200E10E9437
:106EF000452AF5D8A6D9089501E50093322901E085
:106F000000935329ECEDFDE0A4E5B9E200E10E9415
:106F1000452AE5D80091EB28003061F402E00093A7
:106F20005329EBEEFDE0A4E5B9E200E10E94452A19
:106F3000D6D82BC00091EB28E0E0FAE00E94CE28E2
:106F40000E94BE2779F001E00093EB2800E210E0F8
:106F500000939420109395200091EB2800939620A5
:106F60000E94BF1102E000935329E7EFFDE00E9469
:106F700018280091EB280E9460290E94F628E4E579
:106F8000F9E200E10E943028AAD8089500918429EE
:106F90002EC00091EB28003021F404E00093EB2890
:106FA00005C0EBEEF8E200810A95008324C0EBEE09
:106FB000F8E20081039500830091EB28043020F073
:106FC00019F000E00093EB2816C000E210E00093F7
:106FD0009420109395200091EB28009396200E9416
:106FE000BF1100913229007F0093322904C0E4E0F0
:106FF000FAE00E949928089501E000935329E6E001
:10700000FEE0A4E5B9E200E10E94452A68D819D95A
:10701000089501E70093322901E000935329E2E14A
:10702000FEE0A4E5B9E200E10E94452A58D80091AB
:10703000E328002361F002E000935329E1E2FEE03F
:10704000A4E5B9E200E10E94452A49D80BC002E05C
:1070500000935329E8E2FEE0A4E5B9E200E10E94D2
:10706000452A3DD808950091852919C00091E3284B
:107070000E94BE270093E32816C00EE110E00093A3
:107080009720109398200091E328009399200E9464
:10709000ED1100913229007F0093322904C0E2E112
:1070A000FAE00E949928089501E000935329E1E352
:1070B000FEE0A4E5B9E200E10E94452A10D8C1D85B
:1070C00001E000934A29089500919B2800936829C4
:1070D000C3D801E000935329EFE3FEE00E94182893
:1070E000E3E3F9E20E940C280E94F628E4E5F9E2C5
:1070F00000E10E9430280E946F3000914A29003040
:1071000069F402E000935329EBE4FEE0A4E5B9E260
:1071100000E10E94452A0E946F3049C06BD3019163
:1071200010811F930F9370D3C895002D3196C89589
:10713000102D4F915F910423152340E050E00E94F1
:10714000D627D9F002E000935329E8E5FEE00E943B
:10715000182800914A290E9460290E94F628EFE52C
:10716000FEE00E9418280E94F628E4E5F9E200E11A
:107170000E9430280E946F301AC002E00093532909
:10718000E8E5FEE00E94182800914A290E94602943
:107190000E94F628E6E6FEE00E9418280E94F628E3
:1071A000E4E5F9E200E10E9430280E946F30089582
:1071B0000091862953C000914A29003038F031F0FF
:1071C000EAE4F9E200810A95008303C000E100933C
:1071D0004A2948C0EAE4F9E200810395008300915E
:1071E0004A29003120F019F000E000934A293AC002
:1071F00000914A29003031F400913229007F009338
:1072000032292BC0F7D2FF93EF93E091E128F09160
:10721000E228019110811F930F93F6D2C895002D9B
:107220003196C895102D4F915F9104271527512F46
:10723000402FEF91FF9141935083F0D21F2F0E2FDB
:1072400000939A2010939B20D5D201911081009336
:107250009C2010939D200E94DF1204C0E0E2FAE01F
:107260000E949928089501E000935329EDE6FEE07D
:10727000A4E5B9E200E10E94452A0E946F300E9415
:10728000213100E000934B29089501E00093532938
:10729000EEE7FEE0A4E5B9E200E10E94452A0E9483
:1072A0006F3000914B29002369F002E000935329CD
:1072B000E0E9FEE0A4E5B9E200E10E94452A0E946F
:1072C0006F300CC002E000935329E1EAFEE0A4E530
:1072D000B9E200E10E94452A0E946F3008950091B2
:1072E000872913C000914B290E94BE2700934B2988
:1072F00010C000914B29002311F00E943C2D0091F9
:107300003229007F0093322904C0EEE2FAE00E94A5
:107310009928089500E000934C2901E00093532937
:10732000E1EBFEE0A4E5B9E200E10E94452A0E94FB
:107330006F300E94213100E000934B29089501E055
:1073400000935329E2ECFEE0A4E5B9E200E10E94DB
:10735000452A0E946F3000914C29002369F002E019
:1073600000935329E0E9FEE0A4E5B9E200E10E94C0
:10737000452A0E946F300CC002E000935329E1EAD5
:10738000FEE0A4E5B9E200E10E94452A0E946F30C8
:1073900008950091882913C000914C290E94BE27AE
:1073A00000934C2910C000914C29002311F00E9439
:1073B000DF2A00913229007F0093322904C0ECE3D8
:1073C000FAE00E94992808950091322935C00E9460
:1073D000AB3136C017D934C037D932C0F9D930C033
:1073E00043D92EC005DA2CC087DA2AC0E2DA28C0D9
:1073F00063DB26C0ACDB24C023DC22C031DC20C030
:10740000D7DC1EC0E2DC1CC076DC1AC084DC18C0ED
:1074100063DD16C071DD14C0EFDD12C0FADD10C0EF
:1074200043DE0EC051DE0CC01EDF0AC02EDF08C0D6
:1074300071DF06C084DF04C0EAE4FAE00E94992804
:107440000895089500913229007F00933229009118
:107450003229005F0093322900913229003B20F04D
:1074600019F000E000933229089500913229007F3D
:107470000093322900913229003038F031F0009128
:10748000322900510093322903C000E000933229D1
:10749000089500912E290E700093892904E000932D
:1074A0008126E2EDFEE00E94182800912E290E941C
:1074B0004D290E94F628E2E8F6E200E50E94302815
:1074C0000E94DC190091322977C10091892971C08D
:1074D00000913229003019F400E1009332296DC087
:1074E0000091E328002389F00091EA28013021F47B
:1074F00008E00093EA2805C0EAEEF8E200810A9568
:10750000008301E000939C2818C000919C28002370
:1075100021F00091E6280093E4280091E42801304E
:1075200021F408E00093E42805C0E4EEF8E20081CD
:107530000A95008300E000939C2800E00093E9286E
:107540003CC00091E328002389F0EAEEF8E20081D4
:10755000039500830091EA28083020F019F001E03B
:107560000093EA2801E000939C2818C000919C2811
:10757000002321F00091E6280093E428E4EEF8E2ED
:107580000081039500830091E428083020F019F071
:1075900001E00093E42800E000939C2800E00093C1
:1075A000E9280BC001E000939C2800E00093E92843
:1075B00004C0E4EBFAE00E94992802C100918929F5
:1075C00004C053DF06C03EDF04C0E6ECFAE00E94D0
:1075D0009928F6C00091892908C047DF0AC032DF28
:1075E00008C001E20093322904C0E0EDFAE00E94F5
:1075F0009928E6C00091892908C037DF0AC022DF38
:1076000008C001E30093322904C0EEEDFAE00E94C5
:107610009928D6C00091892900937B2986D8D0C0AB
:107620000091892900937C2916D9CAC00091892923
:1076300000937D2988D9C4C00091892900937E29AF
:10764000E6D9BEC00091892900937F295FDAB8C0CE
:107650000091892900938029A4DAB2C00091892978
:1076600008C003DF0AC0EEDE08C001E4009332293F
:1076700004C0ECEEFAE00E949928A2C0009189298A
:107680000093812917DB9CC00091892908C0EDDE99
:107690000AC0D8DE08C001E60093322904C0EAEF30
:1076A000FAE00E9499288CC00091892900938329CF
:1076B000DDDB86C00091892908C0D7DE0AC0C2DEA2
:1076C00008C001E50093322904C0E8E0FBE00E9415
:1076D000992876C0009189290093842957DC70C0CD
:1076E0000091892908C0C1DE0AC0ACDE08C001E7EC
:1076F0000093322904C0E6E1FBE00E94992860C0B3
:107700000091892900938529AEDC5AC0009189290E
:1077100008C0ABDE0AC096DE08C001E8009332293B
:1077200004C0E4E2FBE00E9499284AC00091892944
:10773000009382291ADB44C00091892908C095DE94
:107740000AC080DE08C001E90093322904C0E2E3E8
:10775000FBE00E94992834C0009189290093862972
:1077600027DD2EC00091892908C07FDE0AC06ADEAD
:1077700008C001EA0093322904C0E0E4FBE00E9463
:1077800099281EC00091892900938729A8DD18C077
:107790000091892906C069DE08C001EB00933229F7
:1077A00004C0EEE4FBE00E9499280AC000918929F8
:1077B00000938829EEDD04C0E8E5FBE00E949928EB
:1077C00003DE089500916529112744E559E2040F6D
:1077D000151F2EC000919B2811274EEE58E2040F72
:1077E000151F26C000919B2811274CE350E0040F81
:1077F000151F1EC000919B281127000F111F4BEF72
:1078000058E2040F151F14C000914A291127000FD8
:10781000111F4EE652E0040F151F0AC000919B286D
:107820001127000F111F41E250E0040F151F00C087
:0E784000E02FF12FE093E128F093E228089565
:00000001FF
